:10665C00011900000B01013C0200000301FA0400C7
:10666C00FA0500030A0A5A0B001E0C00FA0D00036F
:10667C000E00040F0164100096120132130AFA1472
:10668C00010215010217010A1801FA1905321A0143
:10669C000A1B01FA1C05321FFFFF20FFFF23011EFE
:1066AC002400642A00FA2B00FA2C50782D003C2E82
:1066BC0000462F001E300064325078330000343214
:1066CC00FA350164360164370150380A643C0064C1
:1066DC003E003C3F000140FFFF411450420A5A4328
:1066EC000AC84405324500B44600FA47013C480349
:1066FC00034C00FA4EFFFF500303510596520A3229
:10670C00530B46540A965601035705465800025936
:10671C000A465A32FA5B010A5C0A325E000A5F00D2
:10672C00FE61FFFF64010F66000267FFFF6A0A3C0F
:10673C006B00006C329673000074000078013279A3
:10674C0001327EFFFF81FFFF84FFFF8500AF8600D3
:10675C00018700FA89010A8A00009900009D0A96B7
:10676C009E00019FFFFFA0FFFFFAFAFA00000B0149
:10677C00013C0200000301FA0400FA0500030A0AB6
:10678C005A0B001E0C00FA0D00030E00040F0164DE
:10679C00100096120132130AFA14010215010217A5
:1067AC00010A1801FA1905321A010A1B01FA1C0513
:1067BC00321FFFFF20FFFF23011E2400642A00FA72
:1067CC002B00FA2C50782D003C2E00462F001E304A
:1067DC0000643250783300003432FA3501643601EB
:1067EC0064370150380A643C00643E003C3F0001B1
:1067FC0040FFFF411450420A5A430AC8440532452F
:10680C0000B44600FA47013C4803034C00FA4EFF23
:10681C00FF500303510596520A32530B46540A9605
:10682C00560101570546580001590A465A32FA5B7F
:10683C00010A5C0A325E000A5F00FE61FFFF640120
:10684C000F66000267FFFF6A0A3C6B00006C329611
:10685C007300007400007801327901327EFFFF81F1
:10686C00FFFF84FFFF85FFFF86FFFF87FFFF890186
:10687C00028A00009900009D0A969E00019FFFFF6E
:10688C00A0FFFFFAFAFA0065006F00790083008D13
:10689C00009700A100AC00B600C000CA00D400DE16
:1068AC0000E800F20058006000680070007800807A
:1068BC0000880090009800A000A800B000B800C1AB
:1068CC0000C800D000D800DF00E600EE00F6004162
:1068DC000047004D00530059005F0065006C0071CB
:1068EC000077007D00830089008F0095009B00A23B
:1068FC0000A700AC00B200B900C000C500CA00D2AD
:0A690C0000D500DD00E100E700EF18
:103A3900900054E0D3940440149007C5E0FEA3E03D
:103A4900FF90665E126A4FE493F59980129007C55C
:103A5900E0FEA3E0FF906778126A4FE493F599902E
:103A690007C5E0FEA3E0FF90665CE493FC74019354
:103A7900FDEFB50507EEB50403754D009007C512B6
:103A89006A362275A71085F97385FA747E017F005D
:103A9900E574126A28E5732FFF50010E8E5A8F5B69
:103AA900900017E0FCA3E0FDEF2DFDEE3CFC8C5CE3
:103AB9008D5D2275A71085F97385FA747E017F00E3
:103AC900E574126A28E5732FFF50010E8E5A8F5B39
:103AD9009000E7E0B40210AC2CAD2DEF2DFDEE3CCB
:103AE900FC8C5C8D5D8016AE5AAF5B900017E0FCD4
:103AF900A3E0FDEF2DFDEE3CFC8C5C8D5D22AE5A02
:103B0900AF5B740C8E048F05FF126A188C5C8D5D97
:103B1900AE5AAF5B740C8E048F05FF126A438C5A40
:103B29008D5BE55B455A6013740CC3955BFFE495A7
:103B39005AFE8E5A8F5B785C126A7CE573A85CB872
:103B49000015D3955D4010E573C3955DFFE4955C61
:103B5900FE8E5C8F5D8010E573243CC3955DFFE4A8
:103B6900955CFE8E5C8F5D757300AE5CAF5D741302
:103B79006F4E600674146F4E7018AE5CAF5D7413AF
:103B89006F4E70057573018003757302755D12754B
:103B99005C00AE5CAF5D74276F4E600674286F4E93
:103BA9007018AE5CAF5D74276F4E70057573018038
:103BB90003757302755D26755C00AE5CAF5D743B81
:103BC9006F4E6006743C6F4E7018AE5CAF5D743B0F
:103BD9006F4E70057573018003757302755D3A75D3
:103BE9005C0022900095E0B40104C2108002D2105A
:103BF900900096E0B40104C2118002D2119000D362
:103C0900E075F0DCA4FFAEF0740A8E048F05FF1294
:103C19006A189007BBECF0A3EDF0A20D40167403EF
:103C29008C068D07126A2874011200399007B9EEC3
:103C3900F0A3EFF07E017F00900091E0126A2890D6
:103C490000D4E08E048F05FF126A18740AFF126A05
:103C5900188D609000DDE075F0DCA4FFAEF0740A09
:103C69008E048F05FF126A189007BFECF0A3EDF0E0
:103C79009000DFE060139000DFE0F5F0741684FF38
:103C89007E00EF9007CDF0800674649007CDF09028
:103C990000D5E0900079F090011FE0900063F0906A
:103CA90000AEE0900065F0900083E0900067F0902E
:103CB9000109E090006CF090016DE090006DF090CA
:103CC900016EE090006EF090016FE090006FF0A23D
:103CD90029B3401690016DE0700C90016EE07006FA
:103CE90090016FE060028002C22974E3900078F0CD
:103CF9009000BEE0B40B0874E3900078F0805A900D
:103D090000BEE0B419129000D4E090687D12008CD6
:103D1900E493900078F080419000BEE0B41E1290C8
:103D290000D4E090689B12008CE493900078F080B6
:103D3900289000BEE0B428129000D4E09068C51223
:103D4900008CE493900078F0800F9000BEE0B446B8
:103D5900089000B5E0900078F09000EEE0FE900049
:103D6900BCE06E600A9000BCE09000EEF0D22890B2
:103D7900007DE0FE9000D7E0B5063390007CE0FEC0
:103D89009000BBE0B5062790007FE0FE9000D9E0E7
:103D9900B5061B90007EE0FE9000E7E0B5060F90A7
:103DA9000080E0FE90008EE06E7003023F0D9000EF
:103DB900E7E06008740790010AF08006740A900130
:103DC9000AF09000D7E0B4020674039000D7F0908F
:103DD900008EE0B4010674009000F4F090008EE0CB
:103DE900B4020674009000D9F090008EE0B4030686
:103DF90074009000E6F09000BBE060147418900025
:103E0900A2F074009006CFF074009006D0F0800CF8
:103E190074009000A2F074189006CFF09000D9E0D9
:103E2900D394014014741990010CF074009006D3D6
:103E3900F074009006D4F0800C740090010CF074BA
:103E4900199006D3F09000BBE0B40214741A9000E4
:103E5900A3F074009006D7F074009006D8F0800C97
:103E690074009000A3F0741A9006D7F09000E7E070
:103E7900701474049006E3F074059006E7F0740674
:103E89009006EBF0802474009006E3F0740090062D
:103E9900E4F074009006E7F074009006E8F074000E
:103EA9009006EBF074009006ECF0D2289000D7E071
:103EB90090007DF09000BBE090007CF09000E7E07E
:103EC90090007EF09000D9E090007FF090008EE0A5
:103ED900900080F090008EE0900064F09000D7E0B0
:103EE900900066F09000C9E0900068F09000E7E06B
:103EF900900069F09000BBE090006AF09000D9E072
:103F090090006BF09000F1E0B40117900023740F5A
:103F1900F0A374FFF0900025E4F0A3F07402900080
:103F2900F1F09000F1E0B40341900025E0FEA3E038
:103F3900FF900023E0FCA3E0FD126A747410126A7A
:103F4900287408120039EF900075F0EF700674FFBD
:103F5900900075F074009000F1F0900024E090005A
:103F690076F0900023E0900077F0900082E09000D6
:103F790043F0900043E02414900044F0900043E0A3
:103F89002428900045F0900044E0D3943C400B90E5
:103F99000044E0C3943C900044F0900045E0D39481
:103FA9003C400B900045E0C3943C900045F09000E4
:103FB90049E4F0900043E064136007900043E0B4E3
:103FC9001420900043E0B413067402900049F09065
:103FD9000043E0B414069000497401F07415900090
:103FE90043F0900043E064276007900043E0B42861
:103FF90020900043E0B427067402900049F0900035
:1040090043E0B428069000497401F07429900043F4
:10401900F0900043E0643B6007900043E0B43C202B
:10402900900043E0B43B067402900049F0900043CD
:10403900E0B43C069000497401F09000437401F02B
:1040490090004AE4F0900044E06413600790004453
:10405900E0B41420900044E0B41306740290004ABE
:10406900F0900044E0B4140690004A7401F074150D
:10407900900044F0900044E064276007900044E019
:10408900B42820900044E0B42706740290004AF056
:10409900900044E0B4280690004A7401F074299015
:1040A9000044F0900044E0643B6007900044E0B4B1
:1040B9003C20900044E0B43B06740290004AF09022
:1040C9000044E0B43C0690004A7401F09000447446
:1040D90001F090004BE4F0900045E0641360079014
:1040E9000045E0B41420900045E0B4130674029032
:1040F900004BF0900045E0B4140690004B7401F0B9
:104109007415900045F0900045E064276007900021
:1041190045E0B42820900045E0B4270674029000D9
:104129004BF0900045E0B4280690004B7401F07400
:1041390029900045F0900045E0643B6007900045F8
:10414900E0B43C20900045E0B43B06740290004B7B
:10415900F0900045E0B43C0690004B7401F09000EB
:10416900457401F0900082E0FE9000E5E02E900099
:104179004DF09000C0E0B4013790004DE075F00FAC
:1041890084AFF07E00EF90004DF0EFB40A06740B97
:1041990090004DF090004DE0B40906740890004D70
:1041A900F090004DE0240F90004EF075510F802BD8
:1041B90090004DE075F00A84AFF07E00EF90004D5D
:1041C900F0EFB40A0690004D7401F090004DE0B490
:1041D9000906740890004DF075510A9000C8E090E6
:1041E9000046F0900046E06414600F900046E064D9
:1041F900286007900046E0B43C06900046E004F0D1
:10420900900046E06413600F900046E06427600761
:10421900900046E0B43B06900046E014F09000465A
:10422900E0D3943C400B900046E0C3943C90004698
:10423900F0900046E02414900047F0900046E024F6
:1042490028900048F0900047E0D3943C400B900040
:1042590047E0C3943C900047F0900048E0D3943C79
:10426900400B900048E0C3943C900048F022C29370
:10427900C294C291C292C287C290E5B554EFF5B516
:10428900E5B554DFF5B5C296C295C2A0C297C2A2E0
:10429900C2A1E5B554BFF5B5E5B5547FF5B5E5B5AA
:1042A90054FBF5B5C213755E469000CBE0700575F9
:1042B9006D028003756D0375550075540090000CEF
:1042C90074FFF0A374DCF0C219C21BC21D74C8903C
:1042D9000037F074C890003BF074C890003FF07547
:1042E9005300755200C20D754600E56FB409037598
:1042F9006F00756300900019E4F0A3F0757010C2A7
:1043090016C217C2189007BBE0FEA3E0FF740312A0
:104319006A2874011200399007B9EEF0A3EFF0C2D0
:1043290002755700755600900010E4F0A3F0C22AF8
:1043390075590075580090008DE075F032A4FDACF8
:10434900F0900021ECF0A3EDF0C23AC212A22EB314
:104359009205A22FB39206A230B39207A231B3926B
:1043690008A232B39209A233B3920AA234B3920BD0
:10437900A235B3920C2275A71085F97385FA747E5C
:10438900017F00E574126A28E5732FFF50010E8E34
:104399005A8F5BAC5CAD5DEF2DFDEE3CFC8C5C8D0A
:1043A9005DD293D294D291E55DF5FBE55CF5FCE530
:1043B9005DF5E9E55CF5EAE55DF5EBE55CF5EC75E0
:1043C900A7002285F97385FA747E017F00E57412CE
:1043D9006A28E5732FFF50010E8E5A8F5B7E017F8D
:1043E90076900106E0126A28AC5AAD5BED2FFFEC1E
:1043F9003EFE8E5C8F5DE55DF5EDE55CF5EE9000CA
:1044090079E4F07412900050F02285F97385FA74FA
:104419007E017F00E574126A28E5732FFF50010EB3
:104429008E5A8F5B9007BBE0FCA3E0FDEF2DFDEEFC
:104439003CFC8C5C8D5DE55DF5FDE55CF5FE2205DA
:104449006422A2DBB340089000D5E0900079F0A285
:10445900DCB34006C296C295C2A075D8402285A792
:104469007275A7109000E7E0B4011DA2D8B340040B
:10447900C293C292A2D9B34004C294C287A2DAB34A
:104489004004C291C2908031A2D8B34002C293A223
:10449900D9B34002C294A2DAB34002C2919000E7B4
:1044A900E0B40215A2DBB34002C292A2DCB340021F
:1044B900C287A2DDB34002C29075D8408572A72297
:1044C900900047E4936406600280FE74C89007C1B7
:1044D900F8E4F0E8A3F075B50075840175A70075D7
:1044E900FFA090004CE4F075C91075A70F75A1C71E
:1044F90075A70075D90075CE0C75A70F75F1FE75F6
:10450900F2FF75F30775F47875A4BA75A5FF75A65A
:104519000775AE0075AFFF75D48175D5FF75D6FFE8
:1045290075D7FF75A70075A20175A14775F80975BB
:10453900D80075D90475DD0975DE0975D84075A7E8
:104549001075D80075D90475DA0975DB0975DC09A8
:1045590075DD0975DE0975DF0975D84075A7007520
:10456900E60875E71075BC0175BE0475BD6C75BEAE
:104579000775BDA075BE0875BD0175BC0075BB1872
:1045890075BC2075BA0875E88075D11375A70F75C4
:10459900E10575E20075C740124277759700759776
:1045A90080740A126A087597C0E5975420700280D2
:1045B900F8758F0275A700D2AF75980075A90C75AB
:1045C900A70F75AB4375ADFB75AC1E75A71075C903
:1045D9001875CA0075CB0075C80475A700758912CE
:1045E900758E04758C00758A00C2A9D28C758D00F0
:1045F900758B00D2ABD28E75EF0675D944C2997509
:1046090009C87508001200E975B5001204E9746358
:104619009007C1F8E4F0E8A3F012037574C8900795
:10462900C1F8E4F0E8A3F07509647508001200E91F
:10463900900064E090008EF090008EE0D3940340E7
:104649000C740090008EF07400900064F0C2219008
:10465900008EE090626DF82828738028A2B4400289
:10466900D221802075A70F75F30F75A700A2A3406B
:1046790002D221800F75A70F75F31775A700A2A4A1
:044689004002D221F8
:0C626D0002466302466502466D02467E52
:10468D00A221B3405E757308E573D3940E501FE5F8
:10469D00739007C1F8E4F0E8A3F0120244750964C1
:1046AD007508001200E97873740126F650DA740269
:1046BD009000CAF0900064E090008EF090008EE0C3
:1046CD00906279F8282873801674009000F4F080B9
:0F46DD000E74009000D9F0800674009000E6F093
:0C6279000246D40246D60246DE0246E68B
:1046EC00D220805C757301E573D39407501FE5737A
:1046FC009007C1F8E4F0E8A3F01202447509647560
:10470C0008001200E97873740126F650DA740190EF
:10471C0000CAF0900064E090008EF090008EE09063
:10472C006285F8282873801674009000F4F0800ECF
:0E473C0074009000D9F0800674009000E6F042
:0C62850002473202473402473C02474403
:10474A00C220900063E090011FF0900064E09000A6
:10475A008EF0900065E09000AEF0900066E0900068
:10476A00D7F0900067E0900083F0900068E0900036
:10477A00C9F0900069E09000E7F090006AE09000CC
:10478A00BBF090006BE09000D9F090006CE09001D3
:10479A0009F090006DE090016DF090006EE09001DC
:1047AA006EF090006FE090016FF090016DE0700C78
:1047BA0090016EE0700690016FE060028004C229E9
:1047CA008002D2299000D4E07006740A9000D4F0D6
:1047DA009000B5E0700674E39000B5F09000BBE07D
:1047EA000490007CF09000BCE09000EEF0123BECEC
:1047FA00E5B54401F5B57406900052F074019000D5
:10480A0053F07403900055F07405900056F0745AF2
:10481A00900057F07405900058F0900054E0B404EA
:10482A00067404900058F07401900059F0740090D6
:10483A00005EF07400900061F074FF900062F07402
:10484A0036900158F07430900159F0742D90015A45
:10485A00F0743690015BF0742B90015CF074489010
:10486A00015DF0746F90015EF0746D90015FF074F9
:10487A0065900160F07420900161F07420900162EB
:10488A00F07433900163F07443900164F07479908A
:10489A000165F0746C900166F09000F0E09000758C
:1048AA00F09000A7E0900076F09000A8E0900077E2
:1048BA00F0A2B6B3920EA2B3B3920FA2A4B39225FA
:1048CA00A2B4B39226A2A3B39227900071E4F07522
:1048DA006F00743A900781F074FD900782F090009F
:1048EA0072E4F09007BBE0FEA3E0FF7403126A28AB
:1048FA0074011200399007B9EEF0A3EFF0756E015A
:10490A00900050E4F0C224756300C214D215C202AA
:10491A00757100C22CD203C22DD204C22ED205C296
:10492A002FD206C230D207C231D208C232D209C24D
:10493A0033D20AC234D20BC235D20CC222C223C22B
:10494A002812009E755F00756B00756100756532EF
:10495A00756600756700756800756900756A00906C
:10496A000019E4F0A3F0756C00D2B2D2A4D2B0D28E
:10497A00B1D2A3D2A7D2A6D2A5D2B790008DE0D346
:10498A0094FA400674FA90008DF07E017F00900040
:10499A0077E0126A28900076E02FFF50010E90000F
:1049AA0023EEF0A3EFF0EFD394FFEE940F400790BD
:1049BA000023E4F0A3F0900075E0700674FF900005
:1049CA0075F09000CAE0D39402400674019000CAC0
:1049DA00F09000CBE07005756D028003756D039051
:1049EA0000CCE0D39401400674009000CCF0900013
:1049FA00D2E0C3940A5006740A9000D2F09000DC08
:104A0A00E0700674019000DCF09000DCE0B4FF0670
:104A1A0074FE9000DCF09000E3E0D394FE4006744C
:104A2A00FE9000E3F0900109E0D39402400674017D
:104A3A00900109F090011FE0D3940140067401909F
:104A4A00011FF074019000E9F074019000EAF0741B
:104A5A00009000F1F0740090010DF07400900111C3
:104A6A00F074299006C7F0742A9006CBF0741B9054
:104A7A0006DBF0741C9006DFF0D29C9000BCE0D3F9
:104A8A009404400674049000BCF0E570D39410407E
:104A9A00037570109006C8E0D3940C400674009019
:104AAA0006C8F09006CCE0D3940C40067400900639
:104ABA00CCF09006D0E0D3940C400674009006D057
:104ACA00F09006D4E0D3940C400674009006D4F01B
:104ADA009006D8E0D3940C400674009006D8F09063
:104AEA0006DCE0D3940C400674009006DCF09006D5
:104AFA00E0E0D3940C400674009006E0F09006E4DF
:104B0A00E0D3940C400674009006E4F09006E8E0C6
:104B1A00D3940C400674009006E8F09006ECE0D3BB
:104B2A00940C400674009006ECF0D2EC75CF01A20A
:104B3A0098B34005C298120646E54D6006A299B39D
:104B4A00B340028005C299120C57E54E6401600514
:104B5A00E54EB4040280D5C28E7E107F00E5641251
:104B6A006A28E58D75F010A4FDACF0EF2DFDEE3C42
:104B7A00FCE58B75F01084FF7E00ED2FFFEC3EFE06
:104B8A008E548F55D28E9000AEE060099000AEE050
:104B9A00C3943D4002805C90001B126A3690001B51
:104BAA00E0FEA3E0FF90001DE0FCA3E0FDEFB505E9
:104BBA0042EEB5043EB21FA20DB3401975E700A23A
:104BCA001FB34008E5B54404F5B58006E5B554FBC6
:104BDA00F5B575E71090001DE0FEA3E0FF90001FF9
:104BEA00E0FCA3E0FDEF2DFDEE3CFC90001DECF097
:104BFA00A3EDF09000BBE060099000BBE0C3940312
:104C0A004002806F122D96A20DB35009900071E0F8
:104C1A00C39423400280069000A5E0F545E545755A
:104C2A00F005A4FFAEF09007C3EEF0A3EFF09000FA
:104C3A0092E0C395614007E55FC39560500790070E
:104C4A00C3E4F0A3F0AE2EAF2F9007C3E0FCA3E0BD
:104C5A00FDEFD39DEE9C4004C2A1800B900071E051
:104C6A00C394325002D2A19000BBE0B40205A2A1C3
:104C7A00B392A29000BBE0B4031C122EB1AE2EAFC9
:104C8A002F9007C3E0FCA3E0FDEFD39DEE9C400408
:104C9A00D2A18002C2A1900096E06009A2B3300FAF
:104CAA0001B3B340028029A2B3300F01B34021A25D
:104CBA00B3301101B3400CA213B34002D212A211B5
:104CCA00B3920FA211B330B301B34004A211920FF1
:104CDA00A2B6300E01B35003025351A2B6300E01F0
:104CEA00B35003025351A2B6301001B3500302511C
:104CFA0095756E00055EA213B3B35013AE54AF554B
:104D0A0090000CE0FCA3E0FDEDC39FEC9E40030283
:104D1A004E41E55E64136005E55EB42709E55E244D
:104D2A0002F55E024E1DE56DB4032EA22AB340229F
:104D3A00E55EB43B03756D01E55EC3943B50069096
:104D4A0000507401F0E55ED3943B40067402900073
:104D5A0050F0755E01D22A805CE56DB40206756D6D
:104D6A0001755E3BE55EB43B05755E0180479000C8
:104D7A0050E07032E55EC3943B50069000507401D7
:104D8A00F0E55ED3943B40067402900050F0E55E75
:104D9A00C3943B5002D224E55ED3943B4002D22412
:104DAA00C296C295C2A09000CBE0B4010512427728
:104DBA008003755E01A212B34005755E01C21290AE
:104DCA0000AEE060099000AEE0C3943D400280432B
:104DDA0090001BE0FEA3E0FF9000AEE08E048F057A
:104DEA00FF126A1874018C068D0712003990001F91
:104DFA00EEF0A3EFF090001FE0F8A3E090001DC8CA
:104E0A00F0A3C8F090001BE4F0A3F0C21FE5B5546C
:104E1A00FBF5B5AE56AF57AC54AD55EF2DFDEE3C94
:104E2A00FC74028C068D071200398E568F57A22405
:104E3A00B34002C224803AAE56AF57AC54AD55EFD8
:104E4A002DFDEE3CFC74018C068D071200398E563E
:104E5A008F57E56DC39402500DAC54AD557418C309
:104E6A009D74159C40028009124277740690005086
:104E7A00F0E55EB43B127403900050F0D224900027
:104E8A00CBE0B40103124277AE58AF59AC54AD55DA
:104E9A00EF2DFDEE3CFC8C588D59AE54AF55EFD337
:104EAA009DEE9C4011900013E0FAA3E0FBEBC39443
:104EBA00E8EA940340028006900013126A369000D2
:104ECA0010E0FEA3E0FFAC54AD55EF2DFDEE3CFC27
:104EDA00900010ECF0A3EDF09000CBE0B40118AE16
:104EEA0054AF557405126A28740112003990000CE7
:104EFA00EEF0A3EFF08011AE54AF557402126A2897
:104F0A0090000CEEF0A3EFF0C28E758D00758B0049
:104F1A00756400755501755400D28EE55E240975D5
:104F2A00F00A84AFF07E00EF4E7075900010E0F842
:104F3A00A3E090000EC8F0A3C8F090000EE0FEA314
:104F4A00E0FFEF4E600B7CA97DB71269168E528F77
:104F5A0053900010E4F0A3F0AE52AF537428BE0091
:104F6A00039F5010E5632FFF50010E7401120039A0
:104F7A008E528F538553639000D2E0A852B8000D29
:104F8A00D395534008E55390004FF080099000D222
:104F9A00E01490004FF0E56D6006755300755200FD
:104FAA00E55E64096005E55EB418099000BBE0603F
:104FBA00031223D29000C0E0B4012F90004DE065A7
:104FCA005E600990004DE0241EB55E08756F00858D
:104FDA005E51801490004EE0655E600990004EE0DC
:104FEA00241EB55E03756F00804390004DE0655E38
:104FFA00600990004DE0241EB55E08756F00855E5D
:10500A0051802A90004DE0240A655E601D90004D93
:10501A00E02414655E601390004DE02428655E600C
:10502A000990004DE02432B55E03756F00A214B3F7
:10503A005006A213B3B340030250EA900087E0B4CB
:10504A000173900109E0B40214120E2690007AE06E
:10505A0075F0BEA4FFAEF08E5C8F5D8056E5677575
:10506A00F00A84FF7E00900581126A4FE0F55B75B5
:10507A005A00AE5AAF5B9000ACE0126A2874648E94
:10508A00048F05FF126A188C5C8D5DE55D90001235
:10509A00F0AE5AAF5B900085E0126A2874648E0401
:1050AA008F05FF126A1874BE8C068D07126A288E45
:1050BA005C8F5D8017900085E075F0BEA4FFAEF0AE
:1050CA008E5C8F5D9000ACE0900012F0E561C394B5
:1050DA00CC5006E55D455C7002800312437FD21412
:1050EA00E56DB40106E55E64096002800975700128
:1050FA009000517401F0E56D60030251909000CE6A
:10510A00E0600D900079E0A852B80006955340027D
:10511A0080409000CEE0B4021F900043E0655E60DC
:10512A000F900044E0655E6007900045E0B55E03BD
:10513A00757003756C00800CC200756C00900019C4
:10514A00E4F0A3F0900079E060067409900050F052
:10515A008034900043E0B55E0B7570019000517485
:10516A0001F08022900044E0B55E0B757001740274
:10517A00900051F08010900045E0B55E097570010D
:10518A007403900051F0A210B3920EA210B330B67D
:10519A0001B35003025351756E01E5B54401F5B5EB
:1051AA007423900071F0A210920EE55ED3944A40E7
:1051BA0014D213E55ED39480400B7403900050F030
:1051CA00D224755E469000D6E0B40107E56AC3941E
:1051DA0014400280091242777413900050F0A22CF6
:1051EA00300301B3501D75E700A22CB34008E5B5A2
:1051FA004408F5B58006E5B554F7F5B575E710A28C
:10520A002C9203A22D300401B3501D75E700A22D84
:10521A00B34008E5B54402F5B58006E5B554FDF599
:10522A00B575E710A22D9204A22E300501B3500FD6
:10523A00A22EB34004D2978002C297A22E9205A250
:10524A002F300601B3500FA22FB34004D2A280021E
:10525A00C2A2A22F9206A230300701B3500FA23089
:10526A00B34004D2A18002C2A1A2309207A2313077
:10527A000801B3501D75E700A231B34008E5B544F3
:10528A0040F5B58006E5B554BFF5B575E710A2310E
:10529A009208A232300901B3501D75E700A232B359
:1052AA004008E5B54480F5B58006E5B5547FF5B507
:1052BA0075E710A2329209A233300A01B3500FA245
:1052CA0033B34004D2928002C292A233920AA23429
:1052DA00300B01B3500FA234B34004D2878002C20C
:1052EA0087A234920BA235300C01B3500FA235B30A
:1052FA004004D2908002C290A235920CE56AC3940F
:10530A00415009740E900050F0124277900058E014
:10531A00FE900054E004C39E4009900054E0D394E8
:10532A0008400974FB900050F012427790005DE04B
:10533A00601590005DE0FE900057E06E600974FE13
:10534A00900050F0124277A224B34006C296C2954A
:10535A00C2A0900106E0600CAE52AF537414BE00B6
:10536A00059F4002804890008EE0906291F82828BC
:10537A0073803BA2B4B35005A226B3400280051243
:10538A0043CCD2268028A2A3B35005A227B3400259
:10539A0080051243CCD2278015A2A4B35005A225BA
:0E53AA00B3400280051243CCD2258002800061
:1062910002537B02537D0253900253A30253B60271
:0262A10053B8F0
:1053B800A216B3B35008900046E0655E60028041D3
:1053C800A201B35006A200B3B34002802E123A8C59
:1053D800E55DF5FBE55CF5FC75A700D293A202B389
:1053E8004002D2929000E7E0B40210123ABCE55DA8
:1053F800F5EDE55CF5EE75A700D292C216D217D28C
:1054080018A217B3B35008900047E0655E600280A9
:1054180041A201B35006A200B3B34002802E123A53
:105428008CE55DF5E9E55CF5EA75A700D294A20282
:10543800B34002D2879000E7E0B40210123ABCE50C
:105448005DF5FDE55CF5FE75A700D287D216C2179B
:10545800D218A218B3B35008900048E0655E600205
:105468008041A201B35006A200B3B34002802E12BD
:105478003A8CE55DF5EBE55CF5EC75A700D291A2F9
:1054880002B34002D2909000E7E0B40210123ABC96
:10549800E55DF5CEE55CF5CF75A700D290D216D2C2
:1054A80017C218E5709062A3F8282873025A109062
:0354B80000BCE055
:0662A3000254B40254B7DE
:1054BB009062D6F8282873121EAE8012121EAE8090
:0E54CB000D121F388008121FE48003121FE428
:0F62D6000254C20254C70254CC0254D10254D60F
:1054D900757002025A10122110122227A23AB34003
:1054E900229000B0E0F56C900081E0256CFE900000
:1054F9004FE075F01E84FC7F00EE2CF53674109099
:105509000050F09007B9E0FEA3E0FF740A126A2880
:1055190090000EE0FCA3E0FD740C8F02FF126A18E4
:105529008D078C038E048A058B061269169007BDB8
:10553900EEF0A3EFF09000D7E0B401087478BE0054
:10554900059F4002800D74789007BDF8E4F0E8A348
:10555900F0801B9007BDE0FEA3E0FF74F0BE0003DE
:105569009F500B74F09007BDF8E4F0E8A3F0E5361E
:1055790070037536019007BDE0FEA3E0FFE5362F05
:10558900FF50010E9007BDEEF0A3EFF07570039088
:035599000051E0DE
:0362A9000254DFBD
:10559C009062E5F82828738019A23B400375700AC5
:1055AC008010A23B400375700B8007A23B40037533
:0255BC00700C71
:0C62E5000255A30255A50255AE0255B7A4
:1055BE00025A109006C8E060031224EA900107E038
:1055CE00B40114900108E0A852B800049553500796
:1055DE00E55FC39560400280097415900050F0029B
:1055EE0056719000BCE0D39402403F900090E024AE
:1055FE0003A852B8000495535009900092E0D39539
:10560E006150028008D2017408900050F090009012
:10561E00E0A852B80005D39553500B900092E024A9
:10562E0003C395615002C2018039900090E02403BB
:10563E00A852B8000495535007E55FC39560400229
:10564E008008D2017408900050F0900090E0A852AB
:10565E00B80005D395535009E560240FC3955F50EC
:10566E0002C2019000D6E07007E56AC394144002AE
:10567E008002D201A2014005757004800A75701077
:10568E00900019E4F0A3F0A20DB34029E56775F080
:10569E000A84FF7E00900581126A4FE0C394695020
:1056AE0005122407800F9007BBE0F8A3E09007B91E
:0C56BE00C8F0A3C8F0025A109000BCE035
:0662AC000255C10256C6B6
:1056CA009062F1F8282873120F108012120F1080BE
:0E56DA000D1210BE80081211708003121170A4
:0F62F1000256D10256D60256DB0256E00256E59F
:1056E8009006CCE060031225C6757005025A1012A8
:1056F80012B07570069006D0E060031226B69006C8
:10570800D4E06003122792025A10900012E060065B
:10571800A20DB3B34002801D900012E02529FFAE10
:105728002850010E8E288F29E55ED39419500690D3
:105738000012E014F01214F67570079006D8E060B5
:105748000312286E9006DCE0600312294A025A1000
:10575800900109E0B40203120E9E1218F575700844
:105768009006E0E06003122A269006E4E060031247
:105778002B02025A10121CB1A20D4015900017E01E
:10578800FEA3E0FF7402126A28900017EEF0A3EF60
:10579800F0A216B35005A217B340028006D216D263
:1057A80017D2187570109006E8E06003122BDE908F
:1057B80006ECE06003122CBA025A10025A1090004C
:1057C80039E0C394465008C2967446900039F09068
:1057D8000049E0B4011DE536240CF5369007BDE01C
:1057E800FEA3E0FF740C2FFF50010E9007BDEEF0F2
:1057F800A3EFF0900049E0B4021DE5362418F53611
:105808009007BDE0FEA3E0FF74182FFF50010E9033
:1058180007BDEEF0A3EFF085365B755A00900043A4
:10582800E0F573123B07E55D900039F0900006E55E
:105838005AF0A3E55BF0E57390003AF0C21A9007BE
:10584800BDE0F55AA3E0F55B900043E0F573123B29
:1058580007E55D900037F0900000E55AF0A3E55B9E
:10586800F0E573900038F0C219E56DB40105757064
:105878000B8003757003025A1090003DE0C39446F4
:1058880050139000D7E0B40104C2968002C2957408
:105898004690003DF090004AE0B4011DE536240C26
:1058A800F5369007BDE0FEA3E0FF740C2FFF500112
:1058B8000E9007BDEEF0A3EFF090004AE0B4021D91
:1058C800E5362418F5369007BDE0FEA3E0FF74180E
:1058D8002FFF50010E9007BDEEF0A3EFF085365B69
:1058E800755A00900044E0F573123B07E55D90009F
:1058F8003DF0900008E55AF0A3E55BF0E5739000F1
:105908003EF0C21C9007BDE0F55AA3E0F55B90009D
:1059180044E0F573123B07E55D90003BF090000210
:10592800E55AF0A3E55BF0E57390003CF0C21BE597
:105938006DB4010575700C8003757003025A1090E0
:105948000041E0C3944650139000D7E0B40104C26C
:10595800968002C2A07446900041F090004BE0B4DB
:10596800011DE536240CF5369007BDE0FEA3E0FFE7
:10597800740C2FFF50010E9007BDEEF0A3EFF090CE
:10598800004BE0B4021DE5362418F5369007BDE05B
:10599800FEA3E0FF74182FFF50010E9007BDEEF034
:1059A800A3EFF085365B755A00900045E0F5731259
:1059B8003B07E55D900041F090000AE55AF0A3E549
:1059C8005BF0E573900042F0C21E9007BDE0F55A07
:1059D800A3E0F55B900045E0F573123B07E55D90A9
:1059E800003FF0900004E55AF0A3E55BF0E5739002
:1059F8000040F0C21DE56DB40103756D00757003BC
:085A080080068004800280008A
:1062B2000256F702571202575802577D0257C3027D
:1062C20057C6025881025947025A0A025A0C025A08
:0462D2000E025A104E
:105A1000900037E0B55E028003025AB2A2194072CC
:105A2000900000E0FEA3E0FFEF4E6021AE56AF57BE
:105A3000900000E0FCA3E0FD120003740C8E048FC4
:105A400005FF126A18900000ECF0A3EDF09000380A
:105A5000E0601A900000E0FEA3E0FFAC56AD57EF07
:105A60002DFDEE3CFC900000ECF0A3EDF090003832
:105A7000E0D39401401A900000E0FEA3E0FFAC5692
:105A8000AD57EF2DFDEE3CFC900000ECF0A3EDF0E7
:105A9000D219AE54AF55900000E0FCA3E0FDEFC377
:105AA0009DEE9C400D124413D296C21974C890000A
:105AB00037F0A219B3B35007900037E0B55E02800B
:105AC0000D124413D29674C8900037F0C21990009A
:105AD00039E0B55E028003025B6DA21A407290004D
:105AE00006E0FEA3E0FFEF4E6021AE56AF579000F8
:105AF00006E0FCA3E0FD120003740C8E048F05FF8A
:105B0000126A18900006ECF0A3EDF090003AE06005
:105B10001A900006E0FEA3E0FFAC56AD57EF2DFD56
:105B2000EE3CFC900006ECF0A3EDF090003AE0D3E0
:105B30009401401A900006E0FEA3E0FFAC56AD577A
:105B4000EF2DFDEE3CFC900006ECF0A3EDF0D21A38
:105B5000AE54AF55900006E0FCA3E0FDEFC39DEE10
:105B60009C400AC2967446900039F0C21AA21AB339
:105B7000B35007900039E0B55E02800AC2967446C1
:105B8000900039F0C21A90003BE0B55E028003023B
:105B90005C33A21B4072900002E0FEA3E0FFEF4ED8
:105BA0006021AE56AF57900002E0FCA3E0FD12006A
:105BB00003740C8E048F05FF126A18900002ECF03B
:105BC000A3EDF090003CE0601A900002E0FEA3E03C
:105BD000FFAC56AD57EF2DFDEE3CFC900002ECF013
:105BE000A3EDF090003CE0D39401401A900002E055
:105BF000FEA3E0FFAC56AD57EF2DFDEE3CFC900050
:105C000002ECF0A3EDF0D21BAE54AF55900002E0D1
:105C1000FCA3E0FDEFC39DEE9C40181244139000DE
:105C2000D7E0B40104D2968002D295C21B74C8900A
:105C3000003BF0A21BB3B3500790003BE0B55E02FF
:105C400080181244139000D7E0B40104D296800269
:105C5000D29574C890003BF0C21B90003DE0B55E49
:105C6000028003025D04A21C4072900008E0FEA3C3
:105C7000E0FFEF4E6021AE56AF57900008E0FCA366
:105C8000E0FD120003740C8E048F05FF126A189059
:105C90000008ECF0A3EDF090003EE0601A900008E0
:105CA000E0FEA3E0FFAC56AD57EF2DFDEE3CFC90BF
:105CB0000008ECF0A3EDF090003EE0D39401401A10
:105CC000900008E0FEA3E0FFAC56AD57EF2DFDEECF
:105CD0003CFC900008ECF0A3EDF0D21CAE54AF55A4
:105CE000900008E0FCA3E0FDEFC39DEE9C40159002
:105CF00000D7E0B40104C2968002C29574469000B9
:105D00003DF0C21CA21CB3B3500790003DE0B55E4D
:105D10000280159000D7E0B40104C2968002C295BB
:105D2000744690003DF0C21C90003FE0B55E0280DA
:105D300003025DD5A21D4072900004E0FEA3E0FFC7
:105D4000EF4E6021AE56AF57900004E0FCA3E0FD9B
:105D5000120003740C8E048F05FF126A1890000461
:105D6000ECF0A3EDF0900040E0601A900004E0FE3B
:105D7000A3E0FFAC56AD57EF2DFDEE3CFC900004C8
:105D8000ECF0A3EDF0900040E0D39401401A9000B5
:105D900004E0FEA3E0FFAC56AD57EF2DFDEE3CFC5A
:105DA000900004ECF0A3EDF0D21DAE54AF5590007E
:105DB00004E0FCA3E0FDEFC39DEE9C4018124413E9
:105DC0009000D7E0B40104D2968002D2A0C21D7424
:105DD000C890003FF0A21DB3B3500790003FE0B55C
:105DE0005E0280181244139000D7E0B40104D296EA
:105DF0008002D2A074C890003FF0C21D900041E024
:105E0000B55E028003025EA6A21E407290000AE008
:105E1000FEA3E0FFEF4E6021AE56AF5790000AE0C0
:105E2000FCA3E0FD120003740C8E048F05FF126AC0
:105E30001890000AECF0A3EDF0900042E0601A9098
:105E4000000AE0FEA3E0FFAC56AD57EF2DFDEE3C9F
:105E5000FC90000AECF0A3EDF0900042E0D3940136
:105E6000401A90000AE0FEA3E0FFAC56AD57EF2DBC
:105E7000FDEE3CFC90000AECF0A3EDF0D21EAE5417
:105E8000AF5590000AE0FCA3E0FDEFC39DEE9C40FF
:105E9000159000D7E0B40104C2968002C2A07446F7
:105EA000900041F0C21EA21EB3B35007900041E023
:105EB000B55E0280159000D7E0B40104C29680025E
:105EC000C2A07446900041F0C21E9000D9E0B40216
:105ED000028003025FE6900073E0D3956650649001
:105EE0000073E0F4042566FE9000DCE08E00F5F01F
:105EF000E884FF7E008F73EFC39410500CEF85731E
:105F0000F0A4FDACF08D7380037573FF900073E017
:105F1000D39573400B900073E0C39573F5718003C4
:105F20007571009000F7E0D3957140069000F7E09E
:105F3000F5719000F8E0C3957150069000F8E0F517
:105F4000718071900073E0C39566FE9000DCE08E76
:105F500000F5F0E884FF7E008F73EFC39410500CBF
:105F6000EF8573F0A4FDACF08D7380037573FF852E
:105F7000735B755A00900073E0255BFFAE5A5001C9
:105F80000E8E5A8F5B74FFBE0009D39F4005855B60
:105F90007180037571FF9000F7E0D3957140069012
:105FA00000F7E0F5719000F8E0C39571500690009D
:105FB000F8E0F571A20DB3B3500D900074E0FE90BF
:105FC00000E4E0D39E5002800A7407900050F0C2B3
:105FD00097801375A710E5CDC395714004C29780D3
:105FE00002D29775A700E56FC39409500AA2EDB3DA
:105FF0004005C2ED123050AE54AF557450C39F747B
:10600000469E400C900072E0C3945A400302626ABC
:10601000A213B340091242777406900050F0A221F7
:10602000B34008E5B54404F5B58006E5B554FBF585
:10603000B5A215B3500EE561D394334007E561C3B3
:1060400094CC40028041900109E0B40214120E2663
:1060500090007AE075F050A4FFAEF08E5C8F5D800A
:106060000F900085E075F050A4FFAEF08E5C8F5D60
:10607000E55D455C6011E5B54401F5B5742390001C
:1060800071F012437FD215900072E0D39401400763
:10609000E561C3941A40028002C2159006C8E06010
:1060A000031224EAA22C300301B35017A22CB340F0
:1060B00008E5B54408F5B58006E5B554F7F5B5A291
:1060C0002C92039006CCE060031225C6A22D30046A
:1060D00001B35017A22DB34008E5B54402F5B580D1
:1060E00006E5B554FDF5B5A22D92049006D0E0600A
:1060F000031226B6A22E300501B3500FA22EB340D4
:1061000004D2978002C297A22E92059006D4E06036
:1061100003122792A22F300601B3500FA22FB340D3
:1061200004D2A28002C2A2A22F92069006D8E060FA
:106130000312286EA230300701B3500FA230B340D3
:1061400004D2A18002C2A1A23092079006DEE060D4
:106150000312294AA231300801B35017A231B340CB
:1061600008E5B54440F5B58006E5B554BFF5B5A2E0
:106170003192089006E0E06003122A26A23230092C
:1061800001B35017A232B34008E5B54480F5B5809D
:1061900006E5B5547FF5B5A23292099006E4E060B9
:1061A00003122B02A233300A01B3500FA233B340C3
:1061B00004D2928002C292A233920A9006E8E06072
:1061C00003122BDEA234300B01B3500FA234B340C4
:1061D00004D2878002C287A234920B9006ECE06062
:1061E00003122CBAA235300C01B3500FA235B340C4
:1061F00004D2908002C290A235920C900072E0C34B
:10620000945A5010E56FB40909900072E004F075DB
:106210006F00803BE56FB40903756F00755500751D
:106220005400758D00758B00756400900071E0C39B
:1062300094325008900071E004F0800674329000AF
:1062400071F0900071E0B43206E5B554FEF5B590FA
:106250000072E0D394014007E56AC3944140028094
:0D62600009740E900050F0124277024B3688
:106300000000010001400160018001A001C001E026
:1063100002000300039603B603D603F4040005004D
:106320000512052405360548055A056C057E0590BD
:1063300005A805C005DE0600061406280646066EFA
:1063400006AE05CF00FF013F015F017F019F01BF46
:1063500001DF01FF02FF039503B503D503F303FF3C
:1063600004FF05110523053505470559056B057D16
:10637000058F05A705BF05CE05F1061306270645BF
:10638000066D06AD06ED05DD0FAA0FA50F9F0F9A4E
:106390000F940F8D0F870F800F780F710F680F60AC
:1063A0000F570F4E0F450F3B0F300F250F1A0F0ED3
:1063B0000F020EF50EE80EDB0ECC0EBE0EAE0E9FDB
:1063C0000E8E0E7D0E6C0E5A0E470E340E200E0CE5
:1063D0000DF70DE20DCB0DB50D9D0D850D6D0D5419
:1063E0000D3A0D200D050CE90CCE0CB10C940C7679
:1063F0000C580C3A0C1B0BFB0BDB0BBB0B9A0B79F1
:106400000B570B350B130AF10ACE0AAB0A870A6445
:106410000A400A1C09F809D409B0098C0967094324
:10642000091F08FB08D608B2088E086A0846082328
:1064300007FF07DC07B9079607730751072F070DFA
:1064400006EC06CA06AA068906690649062A060A4D
:1064500005EC05CD05B0059205750558053C0520F0
:10646000050504EA04CF04B5049C048204690451C0
:1064700004390422040B03F403DE03C803B2039DB2
:10648000038903750361034D033B032803160304CB
:1064900002F202E102D102C002B002A00291028225
:1064A0000273026502570249023C022F02220216C1
:1064B000020901FD01F201E601DB01D001C601BBC9
:1064C00001B101A7019D0194018B01820179017045
:1064D0000168016001580150014801410139013250
:1064E000012B0125011E01180111010B010500FFFF
:1064F00000FA0FA60FA00F990F920F8B0F840F7C3D
:106500000F740F6B0F620F580F4E0F430F380F2C85
:106510000F1F0F120F050EF70EE80ED80EC80EB79C
:106520000EA50E930E800E6C0E580E420E2C0E15FC
:106530000DFD0DE40DCB0DB10D950D790D5D0D3FEC
:106540000D200D010CE10CC00C9E0C7C0C590C357F
:106550000C100BEA0BC40B9E0B760B4F0B260AFD9F
:106560000AD40AAA0A800A550A2A09FF09D409A8E6
:10657000097C0950092508F908CD08A10875084AC1
:10658000081E07F307C8079D07730749072006F78A
:1065900006CE06A6067E06570630060A05E405BFA7
:1065A000059B057705540532051004EF04CE04AEB3
:1065B000048F047104530435041903FD03E203C777
:1065C00003AD0394037B0363034B0334031E0308EF
:1065D00002F302DE02CA02B602A30291027F026D3A
:1065E000025C024C023C022C021D020E020001F26F
:1065F00001E401D701CA01BE01B101A6019A018FD0
:106600000185017A01700166015D0153014A014172
:10661000013901310129012101190112010B010484
:1066200000FD00F700F000EA00E400DE00D900D32E
:1066300000CE00C900C400BF00BA00B500B100AD73
:1066400000A800A400A0009C009900950091008E75
:0C665000008A008700840081007E007B2F
:10009E007547009007C5E4F0A3F075310075300088
:1000AE00754D00754E00C237D23874FE9007C7F8F2
:1000BE00E4F0E8A3F074FE9007C9F8E4F0E8A3F0CA
:1000CE0074FE9007D3F0745A9007D4F0745A9007C8
:1000DE00D5F0D239C22BC23BC23622750B00750A3F
:1000EE0000AE0AAF0BAC08AD09EDC39FEC9E4016F7
:1000FE0074FF126A0875CF01780B740126F650044E
:10010E0018E436F650DB2290004CE0B4AA1C90079F
:10011E0081E0B43C159007C1E0FEA3E0FFEF4E6016
:10012E0009741EBE0004D39F5003020243755D0086
:10013E00755C0075F8099007C1E0FEA3E0FF740737
:10014E006F4E6006740E6F4E7006743A900781F013
:10015E009007C1E0FEA3E0FF7408BE001ED39F40CF
:10016E001A7E017F089007C1E0FCA3E0FD1DBDFFD4
:10017E00011C1200038E5A8F5B801F9007C1E0FE98
:10018E00A3E0FF7408126A6C8F048E057E017F084F
:10019E00CDCCCD1200038E5A8F5BAE5CAF5D740C6E
:1001AE00D39F74019E500302023EA2F9B3407EE536
:1001BE005D455C700375A382AE5CAF5D74016F4EDE
:1001CE00700375A300AE5CAF5D74026F4E700D9040
:1001DE0007C2E075F002A4FDACF08DA3AE5CAF5D7E
:1001EE0074036F4E700375A300AE5CAF5D7403BEF7
:1001FE0000039F5013AC5AAD5BED2FFFEC3EFE900B
:10020E00007D126A4FE0F5A3AE5CAF5DEFB40B0953
:10021E00EEB401057414126A08AE5CAF5DEFB40B58
:10022E0007EEB4010375F80D785C126A7C0201A822
:10023E0090004CE4F022755D00755C0075F8099035
:10024E0007C1E0FEA3E0FF7408BE001ED39F401A54
:10025E007E017F089007C1E0FCA3E0FD1DBDFF01FC
:10026E001C1200038E5A8F5B801F9007C1E0FEA305
:10027E00E0FF7408126A6C8F048E057E017F08CD34
:10028E00CCCD1200038E5A8F5BAE5CAF5D7411D372
:10029E009F74019E5003020374A2F9B3500302032C
:1002AE0071E55D455C700375A3D2AE5CAF5D740104
:1002BE006F4E700375A300AE5CAF5D74026F4E702F
:1002CE000D9007C2E075F002A4FDACF08DA3AE5CFC
:1002DE00AF5D74036F4E700375A300AE5CAF5D74BB
:1002EE00046F4E700375A300AE5CAF5D74056F4E68
:1002FE00700375A300AE5CAF5D74066F4E70037530
:10030E00A300AE5CAF5D74076F4E700375A300AEB5
:10031E005CAF5D74086F4E700375A300AE5CAF5D8D
:10032E007408BE00039F5016AC5AAD5BED2FFFEC68
:10033E003EFE900078126A4FE5A3F075A300AE5C06
:10034E00AF5DEFB41009EEB401057414126A08AE75
:10035E005CAF5DEFB41007EEB4010375F80D785C79
:10036E00126A7C02029722755D00755C0075F809B1
:10037E00AE5CAF5D7417BE0004D39F500302044DF4
:10038E00A2F9B3500302044AE55D455C700375A300
:10039E00D2AE5CAF5D74016F4E700375A300AE5CA0
:1003AE00AF5D74026F4E700D9007C2E075F002A43F
:1003BE00FDACF08DA3AE5CAF5D74036F4E70037534
:1003CE00A300AE5CAF5D74046F4E700375A300AEF8
:1003DE005CAF5D74056F4E700375A300AE5CAF5DD0
:1003EE0074066F4E700375A300AE5CAF5D74076F3D
:1003FE004E700375A300AE5CAF5D74086F4E700354
:10040E0075A300AE5CAF5D7408BE00039F500C90E8
:10041E00005A126A4FE5A3F075A300AE5CAF5D748F
:10042E00166F4E70057414126A08AE5CAF5D7416CA
:10043E006F4E700375F80D785C126A7C02037E2293
:10044E0090004CE0B4AB0280030204E8755D0075C9
:10045E005C0075F809AE5CAF5D7412BE007CD39F74
:10046E004078A2F9B34070E55D455C700375A382D8
:10047E00AE5CAF5D74016F4E700375A300AE5CAFE2
:10048E005D74026F4E700D9007C2E075F002A4FD10
:10049E00ACF08DA3AE5CAF5D74036F4E700375A3AD
:1004AE0000AE5CAF5D7403BE00039F500990005F09
:1004BE00126A4FE0F5A3AE5CAF5D74116F4E70051E
:1004CE007414126A08AE5CAF5D74116F4E700375D2
:1004DE00F80D785C126A7C020463229007D0E4F077
:1004EE0074649007C1F8E4F0E8A3F012037574C8C1
:1004FE009007C1F8E4F0E8A3F074FF90005AF0748E
:10050E00FF90005BF074FF90005CF074009000545C
:10051E00F074FF90005DF0740090005FF074019035
:10052E000060F0900066E0B4371A900063E090002F
:10053E005AF0900064E090005BF0900065E090004F
:10054E005CF080469007D07401F074659007C1F896
:10055E00E4F0E8A3F012037574C89007C1F8E4F054
:10056E00E8A3F0900066E0B4371A900063E09000C4
:10057E005AF0900064E090005BF0900065E090000F
:10058E005CF0800674029007D0F09007D1E4F0740E
:10059E00669007C1F8E4F0E8A3F012037574C890F2
:1005AE0007C1F8E4F0E8A3F0900065E0B4371290CC
:1005BE000063E0900054F0900064E090005DF080E5
:1005CE00769007D17401F074679007C1F8E4F0E8F3
:1005DE00A3F012037574C89007C1F8E4F0E8A3F015
:1005EE00900065E0B43712900063E0900054F090F4
:1005FE000064E090005DF0803E74029007D1F074CC
:10060E00689007C1F8E4F0E8A3F012037574C8907F
:10061E0007C1F8E4F0E8A3F0900065E0B43712905B
:10062E000063E0900054F0900064E090005DF08074
:10063E000674039007D1F022E54E64046006E59936
:10064E0064FF60028031A2374004D2378027E54E26
:10065E00600874E6254E900050F0E54D600874F089
:10066E00254D900050F0E54EB4010280FE754E000F
:10067E00754D00C2378002C237E54E90384AF828D1
:10068E002873754E00E599B4FF03754D01E599B4D5
:10069E00FE03754D02E599B4FD03754D03E599B45E
:1006AE00FC03754D04E599B4FA03754D05E599B44F
:1006BE00FB06754E01124277E599B4F906754E04A4
:1006CE00124277E599D394E54007E599C394F0403B
:1006DE0002801685994F754E027E017F00E54FC34D
:1006EE0094E6126A288E328F339007C5E4F0A3F099
:1006FE00E599D394C44007E599C394E64002802857
:10070E0085994F754E0374E5C3954FF533753200D9
:10071E00AE32AF339063001269F7E493F87401932D
:10072E009007C5C8F0A3C8F0D299020C569000638A
:10073E00E07005A229B3400280429007C5E0FEA3F7
:10074E00E0FF74FFBE00039F5009EFC39446EE9482
:10075E000640119007C5E0FEA3E0FFEFD3946DEEC7
:10076E00940640139007C5E0FEA3E0FF90008112AF
:10077E006A4FE599F0800385997480119007C5E062
:10078E00FEA3E0FF900081126A4FE599F09007C535
:10079E00126A369007C5E0FEA3E0FFEFB40106EE45
:1007AE00B4070280030209FD900781E0B43C028089
:1007BE00030209FDA22950030208E8C29C900063BF
:1007CE00E090011FF0900064E090008EF0900065C4
:1007DE00E09000AEF0900066E09000D7F0900067D9
:1007EE00E0900083F0900068E09000C9F0900069FE
:1007FE00E09000E7F090006AE09000BBF090006B94
:10080E00E09000D9F090006CE0900109F090006D3E
:10081E00E090016DF090006EE090016EF090006F30
:10082E00E090016FF0123BEC900075E09000F0F05C
:10083E00900076E09000A7F0900077E09000A8F08E
:10084E0074639007C1F8E4F0E8A3F074AB90004C29
:10085E00F012044E90004CE4F07464F50975080033
:10086E001200E9A2204039757301E573D394075045
:10087E002DE5739007C1F8E4F0E8A3F074AA900098
:10088E004CF0120115E573C39407500A7464F50910
:10089E007508001200E97873740126F650CC803783
:1008AE00757308E573D3940E502DE5739007C1F858
:1008BE00E4F0E8A3F074AA90004CF0120115E57371
:1008CE00C3940E500A7464F5097508001200E97895
:1008DE0073740126F650CC0209E7C29C90011FE00A
:1008EE00900063F090008EE0900064F09000AEE017
:1008FE00900065F09000D7E0900066F0900083E0E5
:10090E00900067F09000C9E0900068F09000E7E07A
:10091E00900069F09000BBE090006AF09000D9E082
:10092E0090006BF0900109E090006CF07400900064
:10093E006DF0740090006EF0740090006FF07463B0
:10094E009007C1F8E4F0E8A3F074AB90004CF012FD
:10095E00044E90004CE4F07464F509750800120022
:10096E00E9757301E573D394075026E5739007C1BB
:10097E00F8E4F0E8A3F074AA90004CF0120115749C
:10098E0064F5097508001200E97873740126F650B3
:10099E00D3D29C7599FB743C900781F0757308E572
:1009AE0073D3940E5026E5739007C1F8E4F0E8A3D4
:1009BE00F074AA90004CF01201157464F5097508D4
:1009CE00001200E97873740126F650D374C89007AC
:1009DE00C1F8E4F0E8A3F080FE74C89007C1F8E413
:1009EE00F0E8A3F0D29C754E00754D007599FB0290
:1009FE000C569007C5E0FEA3E0FFEF4E70068599FA
:100A0E00317530009007C5E0FEA3E0FF74016F4E14
:100A1E00701BAC30AD31AA32AB33ED2BFBEC3AFA96
:100A2E008A068B07900081126A4FE599F09007C5F0
:100A3E00126A369007C5E0FEA3E0FF74026F4E7097
:100A4E0021AC30AD3174566D4C7006E54F64E660E6
:100A5E00028003124277123BEC854F99754E00755A
:100A6E004D00020C569007C5E0FEA3E0FF900081FA
:100A7E00126A4FE599F09007C5126A369007C5E0E5
:100A8E00FEA3E0FFAC32AD338F028E038C068D07D2
:100A9E009063441269F7E493F9740193FEEAD39ECE
:100AAE00EB994009854F99754E00754D00020C5615
:100ABE009007C5E0FEA3E0FF900081126A4FE59912
:100ACE00F09007C5126A369007C5E0FEA3E0FFEF6F
:100ADE00B40006EEB401028003020C5690005CE0F6
:100AEE00D394C7400B90005CE0C394C8F550801AB5
:100AFE0090005CE0D39463400B90005CE0C3946480
:100B0E00F550800690005CE0F550E55075F002A4BB
:100B1E00FFAEF08F73EF900081126A5AEFFCE0FD8A
:100B2E00EC900084126A5AEDFCE0FDEC2DB55002FB
:100B3E008003020C470FEF900081126A5AE573FF93
:100B4E00E0FCEF900085126A5AECFFE0FCEFC39CCC
:100B5E00B550028003020C47E573900083126A5A67
:100B6E00E573FFE0FCEF900086126A5AECFFE0FCA2
:100B7E00EF2CB550028003020C47E57390008712EC
:100B8E006A5AE0C39550900063F0E57390008812A6
:100B9E006A5AE0C39550900064F0E5739000891294
:100BAE006A5AE0C39550900065F07400900066F0AC
:100BBE0074FF900067F0E57390008B126A5AE0C3E1
:100BCE009550900068F0E57390008C126A5AE0C35D
:100BDE009550900069F0E57390008D126A5AE0C34B
:100BEE00955090006AF0E57390008A126A5AE0C33D
:100BFE0095509007C1F8E4F0E8A3F074AB90004C68
:100C0E00F012044E7464F5097508001200E990079D
:100C1E00C1126A3612044E7464F50975080012008A
:100C2E00E99007C1126A3612044E7599F97464F58B
:100C3E00097508001200E980FE7599FF7464F509C4
:080C4E007508001200E980FEA8
:0F384A0002069002073B020A00020A73020ABE3E
:100C560022E54D903859F8282873020D699007C58A
:100C6600E0FEA3E0FF900052126A4FE0F59990076C
:100C7600C5126A369007C5E0FEA3E0FF74116F4EF9
:100C86007003754D00020D69856E99020D69900716
:100C9600C5E0FEA3E0FF900081126A4FE0F599EFF0
:100CA600B40107EEB40703754D009007C5126A3606
:070CB600020D699007C6E082
:0F385900020C60020C63020C8E020C94020CB97C
:100CBD00903A0CF8282873855399020D5E855F993B
:100CCD00020D5E856199020D5E856599020D5E8549
:100CDD006799807D85689980788569998073856A23
:100CED0099806E90001AE0F5998066A238B340079E
:100CFD007599FAC2388041A228B3400575990F80C5
:100D0D00359007D0E0600A9007D0E024DCF599809B
:100D1D00169007D1E0600A9007D1E024DEF59980A6
:100D2D0006900050E0F599900050E4F09007D0E463
:100D3D00F09007D1E4F0C2288017856B9980128559
:100D4D006699800D856C9980087599FC8003754DA9
:010D5D000095
:103A0C00020CC4020CCA020CD0020CD6020CDC0252
:103A1C000CE1020CE6020CEB020CF0020CF8020DAD
:0D3A2C0047020D4C020D51020D56020D5BBC
:0B0D5E009007C5126A368003123A3974
:03386800020D66E8
:100D690022E537255BFFAE5A50010E900081126AC9
:100D79004FE0F538E537255BFFAE5A50010E0FBF3E
:100D890000010E900081126A4FE0F539853F3BE57D
:100D990038B539058538378041E539D39538401D4F
:100DA900E539C39538853AF0A4FFAEF0E53B8E04EA
:100DB9008F05FF126A18ED2538F537801DE538C310
:100DC9009539853AF0A4FFAEF0E53B8E048F05FF17
:100DD900126A18EDF4042538F53722E539D3953828
:100DE900401DE539C39538853AF0A4FFAEF0E53BDF
:100DF9008E048F05FF126A18ED2538F537801DE539
:100E090038C39539853AF0A4FFAEF0E53B8E048FDF
:100E190005FF126A18EDF4042538F537229000878A
:100E2900E0B40170E56775F00A84FF7E008F37E54D
:100E39006775F00A84ADF07C008D3A753F0A755AE2
:100E490005755B24E537C394115005120D6A8006B8
:100E59009005B6E0F537E53790007AF0E56775F06B
:100E69000A84FF7E008F37E56775F00A84ADF07C50
:100E7900008D3A753F0A755A05755B5AE537C39473
:100E8900115005120D6A80069005ECE0F537E5373B
:100E9900900012F022900087E0B4016AE56775F0CE
:100EA9000A84FF7E008F37E56775F00A84ADF07C10
:100EB900008D3A753F0A755A05755B36E537C39457
:100EC900115005120D6A80069005C8E0F53785377F
:100ED9004BE56775F00A84FF7E008F37E56775F08B
:100EE9000A84ADF07C008D3A753F0A755A05755B29
:100EF90048E537C394115005120D6A80069005DA4A
:100F0900E0F53785374C22E55F75F00484FF7E00F4
:100F19008F37E55F75F00484ADF07C008D3A753F3D
:100F290004755A01755B00E537C3943F5005120DEE
:100F39006A80069001C0E0F5378537297528009049
:100F4900004FE075F020A4FFAEF09000D2E08E04CF
:100F59008F05FF126A188D379000BAE0D3955F505C
:100F6900030210169000DEE0D3955F4010ED90016A
:100F7900C1126A5AE0F52B752A000210139000A9D4
:100F8900E0D3955F4043E5379001C1126A5AE0F515
:100F990038E5379001E1126A5AE0F5399000DEE050
:100FA900F404255FF53A9000A9E0FE9000DEE0F434
:100FB900042EF53BE538B539058538378003120D20
:100FC900E485372B752A008041E5379001E1126AE3
:100FD9005AE0F538E537900201126A5AE0F539907E
:100FE90000A9E0F404255FF53A9000BAE0FE90000C
:100FF900A9E0F4042EF53BE538B539058538378085
:1010090003120DE485372B752A000210BD9000E10B
:10101900E0D3955F5011E537900241126A5AE0F525
:101029002B752A000210BD9000AAE0D3955F5043AA
:10103900E537900221126A5AE0F538E53790024106
:10104900126A5AE0F5399000AAE0F404255FF53AEE
:101059009000E1E0FE9000AAE0F4042EF53BE538AB
:10106900B539058538378003120DE485372B752A84
:10107900008041E537900201126A5AE0F538E537F8
:10108900900221126A5AE0F5399000BAE0F4042579
:101099005FF53A9000AAE0FE9000BAE0F4042EF55C
:1010A9003BE538B539058538378003120DE48537B6
:1010B9002B752A00229000F2E0F53C753F11755A14
:1010C90002755B00AE52AF53E53C75F00FA4FDAC61
:1010D900F0EDD39FEC9E4021E53C8E048F05FF1275
:1010E9006A18ED75F010A4FFAEF0E55F75F0118494
:1010F900FD7C00ED2FF53D800EE55F75F01184FF55
:101109007E00EF24F0F53D853D37E55F75F01184EC
:10111900AFF07E008F3A120D6A85373EAE52AF535B
:101129009000F2E075F00FA4FDACF0EDD39FEC9EBA
:101139004028755A02755B10853D37120D6A853E48
:1011490038853739AE52AF53E53C8E048F05FF120F
:101159006A438D3A853C3B120DE485372975280091
:10116900752B64752A00229000F2E0F53C753F1159
:10117900755A02755B00AE52AF53E53C75F00FA48A
:10118900FDACF0EDD39FEC9E4021E53C8E048F052C
:10119900FF126A18ED75F010A4FFAEF0E56175F065
:1011A9001184FD7C00ED2FF53D800EE56175F01190
:1011B90084FF7E00EF24F0F53D853D37E56175F04C
:1011C9001184AFF07E008F3A120D6A85373EAE5218
:1011D900AF539000F2E075F00FA4FDACF0EDD39F92
:1011E900EC9E4028755A02755B10853D37120D6AD1
:1011F900853E38853739AE52AF53E53C8E048F05AD
:10120900FF126A438D3A853C3B120DE485372975F7
:101219002800E56B6017E56BC394FE50109000E65B
:10122900E0B402099000D4E0D3940B50028017AEC9
:1012390028AF29E56B126A2874E78E048F05FF121F
:101249006A188C288D299000BCE0B40453E55F75B9
:10125900F00484FF7E008F37E55F75F00484ADF0FC
:101269007C008D3A753F04755A01755B00E537C3FB
:10127900943F5005120D6A80069001C0E0F537AE23
:1012890028AF29E537126A2874648E048F05FF1286
:101299006A18AE28AF29EF2DFDEE3CFC8C288D296C
:1012A900752B64752A0022900087E0B40146E56732
:1012B90075F00A84FF7E008F37E56775F00A84AD03
:1012C900F07C008D3A753F0A755A05755B00E53764
:1012D900C394115005120D6A8006900592E0F53706
:1012E900AE2AAF2BE5372FFF50010E7464126A6CDA
:1012F9008E2A8F2B900088E0B40146E56875F00AC4
:1013090084FF7E008F37E56875F00A84ADF07C00B4
:101319008D3A753F0A755A05755B6CE537C39411AB
:101329005005120D6A80069005FEE0F537AE2AAF2A
:101339002BE5372FFF50010E7464126A6C8E2A8FC9
:101349002B900097E0B40249E56AC3944175F00512
:1013590084FF7E008F37E56A75F00584ADF07C0067
:101369008D3A753F05755A06755B00E537C39413C9
:101379005005120D6A8006900694E0F537AE2AAF43
:101389002BE5372FFF50010E7464126A6C8E2A8F79
:101399002B9000D9E0B40202800302144FE55F7577
:1013A900F01584FF7E008F37E55F75F01584ADF089
:1013B9007C008D3A753F15755A03755BF4E537C3A3
:1013C900940B5005120D6A8006900480E0F537E50C
:1013D9003775F0FFA4FFAEF09000DAE08E048F05B8
:1013E900FF126A18ED900073F0E56675F078A4FFB6
:1013F900AEF074FF8E048F05FF126A188C5A8D5B4C
:1014090074028C068D071200398F37AC5AAD5B74A4
:1014190004FF126A438D3A753F04755A06755B28B5
:10142900E537C3941D5005120D6A80069006C6E083
:10143900F537AE2AAF2BE5372FFF50010E74641232
:101449006A6C8E2A8F2B900086E0B4025DE5617587
:10145900F064A4FFAEF074081200398E5C8F5D74DD
:10146900058E048F05FF126A188D37AE5CAF5D7467
:10147900058E048F05FF126A438D3A753F05755A2B
:1014890005755BDEE537C394135005120D6A8006B6
:10149900900672E0F537AE2AAF2BE5372FFF5001E2
:1014A9000E7464126A6C8E2A8F2B9000C8E0703C0F
:1014B90090004FE075F00584FF7E008F3790004F54
:1014C900E075F00584ADF07C008D3A753F05755ADD
:1014D90005755BC0E537C3941D5005120D6A80067A
:1014E90090065EE0F537E53790007BF02290008F9B
:1014F900E0B401179007CCE0252BFFAE2A50010E6E
:101509009000E3E0126A6C8E2A8F2B900107E0B4F9
:101519000114900108E0A852B8000495535007E55A
:101529005FC39560400280129000B1E0252BFFAEA9
:101539002A50010E8E2A8F2B802F90008FE0B40342
:1015490016A22BB3B350109007CFE0C39405A8524D
:10155900B800069553400280109000B1E0252BFF9A
:10156900AE2A50010E8E2A8F2B900089E0B4020218
:1015790080030218F490008CE0602FE567D394464D
:101589004028900013E0FEA3E0FF9000C7E075F04B
:1015990003A4FDACF0EFD39DEE9C400E9000EBE070
:1015A900A852B80005D3955350030218F49000BC13
:1015B900E0B40302800302175885615B755A0090F5
:1015C9000093E0A852B800049553500E900094E09F
:1015D900A85AB80005D3955B5003021755E5617504
:1015E900F002A4FFAEF074158E048F05FF126A187D
:1015F9008C068D07900611126A4FFEE0FFEE9000EF
:101609008BE0FEEF8E0088F0A4FFAEF074648E04C8
:101619008F05FF126A188C5A8D5B90004FE075F0A8
:1016290018A4FFAEF09000D2E08E048F05FF126A75
:10163900188C068D07900629126A4FAE5AAF5BE0E7
:10164900126A2874648E048F05FF126A188C5A8DE9
:101659005BE565A85AB80077D3955B4072E565C329
:10166900955BFFE4955AFE8E5A8F5B7428BE000382
:101679009F500C755B28755A00740D900050F0AEA0
:101689005AAF5B90008CE0126A2874288E048F058B
:10169900FF126A188C5A8D5BAE28AF29740A8E0422
:1016A9008F05FF126A188D068C07AC5AAD5BCFCE39
:1016B900CF120003740A8E048F05FF126A188C5A20
:1016C9008D5BAE28AF29126A748E288F29807DE53B
:1016D90065A85AB80004955B5072AE5AAF5BE565D0
:1016E900126A6C8E5A8F5B7428BE00039F500C756A
:1016F9005B28755A00740D900050F0AE5AAF5B909C
:10170900008CE0126A2874288E048F05FF126A186B
:101719008C5A8D5BAE28AF29740A8E048F05FF128F
:101729006A188D068C07AC5AAD5BCFCECF12000379
:10173900740A8E048F05FF126A188C5A8D5BAE28C5
:10174900AF29EF2DFDEE3CFC8C288D290218F49071
:1017590000D4E0855FF0A4FFAEF07405126A287426
:10176900071200398E5A8F5B900093E0A852B80097
:101779000495535012900094E075F002A4FDACF06A
:10178900EFC39DEE9C40030218F4E55F75F00B84EE
:10179900FF7E00900611126A4FFEE0FFEE90008B6B
:1017A900E0FEEF8E0088F0A4FFAEF074648E048F23
:1017B90005FF126A188C5A8D5B90004FE075F0187E
:1017C900A4FFAEF09000D2E08E048F05FF126A18D4
:1017D9008C068D07900629126A4FAE5AAF5BE0124C
:1017E9006A2874648E048F05FF126A188C5A8D5BFF
:1017F900E565A85AB80077D3955B4072E565C3954E
:101809005BFFE4955AFE8E5A8F5B7428BE00039FD6
:10181900500C755B28755A00740D900050F0AE5A43
:10182900AF5B90008CE0126A2874288E048F05FF44
:10183900126A188C5A8D5BAE28AF29740A8E048FF0
:1018490005FF126A188D068C07AC5AAD5BCFCECF57
:10185900120003740A8E048F05FF126A188C5A8DC0
:101869005BAE28AF29126A748E288F29807DE565C1
:10187900A85AB80004955B5072AE5AAF5BE5651281
:101889006A6C8E5A8F5B7428BE00039F500C755B7F
:1018990028755A00740D900050F0AE5AAF5B900055
:1018A9008CE0126A2874288E048F05FF126A188C3E
:1018B9005A8D5BAE28AF29740A8E048F05FF126A10
:1018C900188D068C07AC5AAD5BCFCECF12000374CE
:1018D9000A8E048F05FF126A188C5A8D5BAE28AFE9
:1018E90029EF2DFDEE3CFC8C288D29229000E7E0A4
:1018F900B4026AE55F75F00884FF7E008F37E55F03
:1019090075F00884ADF07C008D3A753F08755A0171
:10191900755BE0E537C3943F5005120D6A80069068
:101929000280E0F53785372D752C00AE2CAF2DAC34
:101939002AAD2B12000374648E048F05FF126A18F6
:101949008C2C8D2D900084E08C068D07126A2874EA
:10195900648E048F05FF126A188C2C8D2DAE28AF6A
:1019690029AC2AAD2B12000374648E048F05FF1273
:101979006A188C288D29900084E08C068D07126ADC
:101989002874648E048F05FF126A188C288D29A289
:101999000D401DAE52AF537405BE00039F5002D2D5
:1019A9000DE561D394CC4008D2017411900050F038
:1019B9009000E6E0B402089000D4E0640B60028075
:1019C90035AE28AF29E56B126A2874E78E048F05B6
:1019D900FF126A188C288D299000E7E0B40217AE2F
:1019E9002CAF2DE56B126A2874E78E048F05FF1260
:1019F9006A188C2C8D2D9000A6E05402601B900073
:101A09009DE0A852B80012D39553400DA20DB3B36F
:101A19005007E561C3949A40028028AE34AF3590EF
:101A2900009BE075F002A4FDACF0EF2DFDEE3CFC4F
:101A390074022DFD50010CE561BC0007D39D4003E4
:101A4900754301856135753400E5437003021B3820
:101A59009000F9E0C395435003021B2A900109E065
:101A6900C394025076E56775F00A84FF7E009005FD
:101A790081126A4FE0F55B755A00AE5AAF5B900070
:101A89009CE0126A2874648E048F05FF126A188C10
:101A99005C8D5D9000F9E004C395438C068D0712B7
:101AA9006A289000F9E08E048F05FF126A188C5C91
:101AB9008D5DAE28AF29EF2DFDEE3CFC8C288D29DC
:101AC9009000E7E0B40212AE2CAF2DAA5CAB5DEF3B
:101AD9002BFBEE3AFA8A2C8B2D80469000F9E00414
:101AE900C39543854BF0A4FFAEF09000F9E08E0456
:101AF9008F05FF126A188C5C8D5DAE28AF29EF2D1A
:101B0900FDEE3CFC8C288D299000E7E0B40212AE72
:101B19002CAF2DAA5CAB5DEF2BFBEE3AFA8A2C8B2E
:101B29002D05439000F9E0C3954350037543009098
:101B390000A6E05401601B90009AE0A852B8001278
:101B4900D39553400DA20DB3B35007E55FC394CCB1
:101B590040028025900098E075F003A4FFAEF0E5FF
:101B6900402FFF50010E74032FFF50010EE55FBE99
:101B79000007D39F4003754401855F40E544700326
:101B8900021C6B9000FAE0C395445003021C5D905F
:101B99000109E0C394025076E56775F00A84FF7E77
:101BA90000900581126A4FE0F55B755A00AE5AAF95
:101BB9005B900099E0126A2874648E048F05FF1205
:101BC9006A188C5C8D5D9000FAE004C395448C061C
:101BD9008D07126A289000FAE08E048F05FF126AB9
:101BE900188C5C8D5DAE28AF29EF2DFDEE3CFC8C89
:101BF900288D299000E7E0B40212AE2CAF2DAA5C23
:101C0900AB5DEF2BFBEE3AFA8A2C8B2D80469000C8
:101C1900FAE004C39544854CF0A4FFAEF09000FAB5
:101C2900E08E048F05FF126A188C5C8D5DAE28AFBB
:101C390029EF2DFDEE3CFC8C288D299000E7E0B4BE
:101C49000212AE2CAF2DAA5CAB5DEF2BFBEE3AFA7C
:101C59008A2C8B2D05449000FAE0C39544500375F6
:101C690044009000FCE02529FFAE2850010E8E2883
:101C79008F299000ABE0A828B80004952950099055
:101C890000ABE0F5297528009000E7E0B4020D905B
:101C990000ABE0A82CB80006952D40028009900001
:101CA900ABE0F52D752C00229000E7E0B40102802D
:101CB90003021DBCA20DB35003021DBA9000B2E08D
:101CC900B40168AE28AF29AC52AD53120003743C7D
:101CD9008E048F05FF126A189000C2E0BC00109DA7
:101CE900400D9000C4E0A828B8000495295002D2FC
:101CF90002AE28AF29AC52AD53120003743C8E04D6
:101D09008F05FF126A189000C2E0C3940ABC00153F
:101D1900D39D40119000C4E0C39405A828B80005DC
:101D2900D3952950028002C2028068AE28AF29AC3F
:101D390052AD5312000374788E048F05FF126A188E
:101D49009000C2E0BC00109D400D9000C4E0A8289E
:101D5900B8000495295004D2028038AE28AF29ACC6
:101D690052AD5312000374788E048F05FF126A185E
:101D79009000C2E0C3940ABC0015D39D40119000A5
:101D8900C4E0C39405A828B80005D395295002805A
:101D990002C202A202B34019AE28AF299000C3E0E3
:101DA900126A2874648E048F05FF126A188C288DB4
:101DB900298002C202A200B34006A201B3B35009AE
:101DC900900019E4F0A3F08024AE28AF297400D361
:101DD9009F74019E400C900019E528F0A3E529F0B5
:101DE900800B74FF900019F8E4F0E8A3F09000C9A3
:101DF900E0D39402400C9000B4E07006A20DB3B396
:101E09004002801AAE28AF297402126A288E288FE0
:101E190029AE2CAF2D7402126A288E2C8F2D9000BA
:101E2900B2E0B4011AAE28AF297402126A288E28CA
:101E39008F29AE2CAF2D7402126A288E2C8F2DAEED
:101E490028AF29745E126A28740A8E048F05FF125E
:101E59006A188C288D299000E7E0B40217AE2CAFE0
:101E69002D745E126A28740A8E048F05FF126A188F
:101E79008C2C8D2DAE28AF297402BE000AD39F4049
:101E890006752902752800AE2CAF2D7402BE000A12
:101E9900D39F4006752D02752C00900017E528F098
:101EA900A3E529F02290004FE0900381126A5AE0DD
:101EB900F54175426490004FE0FE9000BDE0D39E6D
:101EC9004037E55F75F00884FF7E008F37E55F7561
:101ED900F00884ADF07C008D3A753F08755A03759A
:101EE9005B96E537C3941F5005120D6A800690046E
:101EF90036E0F5378537428035E55F75F00884FFB0
:101F09007E008F37E55F75F00884ADF07C008D3A6F
:101F1900753F08755A03755BB6E537C3941F5005BD
:101F2900120D6A8006900456E0F5378537422290F3
:101F390000F3E0F53C753F11755A04755B00AE522C
:101F4900AF53E53C75F00FA4FDACF0EDD39FEC9ECB
:101F59004021E53C8E048F05FF126A18ED75F010DB
:101F6900A4FFAEF0E55F75F01184FD7C00ED2FF55F
:101F79003D800EE55F75F01184FF7E00EF24F0F5DA
:101F89003D853D37E55F75F01184AFF07E008F3AEE
:101F9900120D6A85373EAE52AF539000F3E075F0EB
:101FA9000FA4FDACF0EDD39FEC9E4028755A047543
:101FB9005B10853D37120D6A853E38853739AE523B
:101FC900AF53E53C8E048F05FF126A438D3A853C79
:101FD9003B120DE4853741754264229000F3E0F528
:101FE9003C753F11755A04755B00AE52AF53E53C21
:101FF90075F00FA4FDACF0EDD39FEC9E4021E53CBC
:102009008E048F05FF126A18ED75F010A4FFAEF06B
:10201900E56175F01184FD7C00ED2FF53D800EE53D
:102029006175F01184FF7E00EF24F0F53D853D37A1
:10203900E56175F01184AFF07E008F3A120D6A8563
:10204900373EAE52AF539000F3E075F00FA4FDACEC
:10205900F0EDD39FEC9E4028755A04755B10853DC1
:1020690037120D6A853E38853739AE52AF53E53C94
:102079008E048F05FF126A438D3A853C3B120DE4AD
:102089008537417542649000BCE0B4047990004FF3
:10209900E0FE9000BDE0D39E4037E55F75F008840F
:1020A900FF7E008F37E55F75F00884ADF07C008D09
:1020B9003A753F08755A03755B96E537C3941F5007
:1020C90005120D6A8006900436E0F537853742809F
:1020D90035E55F75F00884FF7E008F37E55F75F0A1
:1020E9000884ADF07C008D3A753F08755A03755B1D
:1020F900B6E537C3941F5005120D6A800690045641
:10210900E0F53785374222900087E0B4013BE56767
:1021190075F00A84FF7E008F37E56775F00A84AD94
:10212900F07C008D3A753F0A755A05755B12E537E3
:10213900C394115005120D6A80069005A4E0F53785
:10214900E5422537C39464F542900088E0B4013B29
:10215900E56875F00A84FF7E008F37E56875F00A37
:1021690084ADF07C008D3A753F0A755A05755B7E22
:10217900E537C394115005120D6A8006900610E0E8
:10218900F537E5422537C39464F542E5412542F523
:102199003690008FE0B402109007CBE02536FE9010
:1021A90000E3E0F4042EF5369000E6E0D394014014
:1021B90040E56BC394E7501D74E7C3956BFE900728
:1021C900CDE08E00F5F0E884FF7E008F37E53625F7
:1021D90037F536801CE56BC394E7FE9007CDE08E9A
:1021E90000F5F0E884FF7E008F37E536C39537F5B3
:1021F90036A20D4006E5412464F536E536D39464EC
:102209004009E536C39464F53680037536009000BD
:10221900BFE0C3953650069000BFE0F53622D200E4
:10222900900079E0A852B800049553504190007984
:10223900E0A852B800049553500375360F90007901
:10224900E004A852B800049553500375360A90006B
:1022590079E02402A852B800049553500575360553
:10226900C200900079E060067409900050F0C23B0A
:102279007E017F009000C5E0126A289000D4E08EAC
:10228900048F05FF126A18E55FBC0017D39D401340
:102299009000CEE0B40204D23B8002C200740A90DE
:1022A9000050F09000C6E0C3956750159000D8E043
:1022B900A852B8000495535002C200740B90005004
:1022C900F0E567C39464501D90011EE0600D900114
:1022D9001EE0A852B80006955340028008C2007457
:1022E9000B900050F0A2004003753605900107E0FD
:1022F900B40114900108E0A852B80004955350079E
:10230900E55FC39560400280089000B0E0F5368033
:102319003A90008FE0B40306A22BB3B34002802B9E
:102329009007CFE0C39405A852B800049553500C08
:102339009000B0E0F536740C900050F09007CFE0B3
:10234900A852B8000495535002C20085366C90001B
:1023590081E02536FE90004FE075F01E84FC7F0079
:10236900EE2CF5362290004FE075F00584FF7E00D3
:102379008F3790004FE075F00584ADF07C008D3A01
:10238900753F05755A03755BD69000D2E01475F058
:102399000584FF7E00E537BE00039F5005120D6AD4
:1023A900800BE537900457126A5AE0F537E5379004
:1023B90007CEF09007CEE0FE9000C1E0C39E500822
:1023C9009000C1E09007CEF022E56775F00A84FF1E
:1023D9007E00900581126A4FE0F546E546D3946484
:1023E9004010E546C3946475F00F84FF7E008F4664
:1023F90080037546009000A4E02546F5462290002A
:10240900BCE0C3940350269007BBE0FEA3E0FF7431
:1024190004120039E55F126A28740F8E048F05FFD4
:10242900126A189007B9ECF0A3EDF080249007BB6D
:10243900E0FEA3E0FF7404120039E561126A287412
:102449000F8E048F05FF126A189007B9ECF0A3EDFF
:10245900F0900097E0B40262E56AC3944175F00513
:1024690084FF7E008F37E56A75F00584ADF07C0046
:102479008D3A753F05755A06755B14E537C3941790
:102489005005120D6A80069006A8E0F5379007B945
:10249900E0FEA3E0FF740A8E048F05FF126A18E5B7
:1024A900378C068D07126A28740A8E048F05FF126D
:1024B9006A189007B9ECF0A3EDF09007B9E0FEA314
:1024C900E0FF9007BFE0FCA3E0FDEDD39FEC9E4049
:1024D9000F9007BFE0F8A3E09007B9C8F0A3C8F0D0
:1024E900229006C8E090386BF8282873804C8553F1
:1024F9007380479000D4E0855FF0A4FFAEF07408C4
:102509001200398F738033856173802E85677380DC
:10251900298568738024856973801F856A73801A89
:10252900856B7380158566738010856573800B854F
:0A2539006C73800690001AE0F57341
:10386B000224F50224F70224FC022510022515027E
:10387B00251A02251F02252402252902252E0225A1
:07388B003302253802253D40
:102543009006C9E0FE9006CAE0D39E404B9006C8B1
:10255300E0B404189006CAE0C395735002D22C90DD
:1025630006C9E0D395734002C22C802A9006C9E0C5
:10257300C3957350099006CAE0D395735002800245
:10258300D22C9006C9E0D3957350099006CAE0C3D4
:1025930095735002C22C802A9006C9E0D3957340EC
:1025A300099006CAE0C3957340028002C22C9006CC
:1025B300C9E0C3957340099006CAE0D395734002FE
:1025C300D22C229006CCE0903892F8282873804CC5
:1025D30085537380479000D4E0855FF0A4FFAEF08D
:1025E30074081200398F738033856173802E856779
:1025F3007380298568738024856973801F856A7356
:10260300801A856B7380158566738010856573806A
:0C2613000B856C73800690001AE0F573D4
:103892000225D10225D30225D80225EC0225F10208
:1038A20025F60225FB02260002260502260A02262A
:0738B2000F02261402261983
:10261F009006CDE0FE9006CEE0D39E405F9006CCB4
:10262F00E0B404189006CEE0C395735002D22D90FB
:10263F0006CDE0D395734002C22D803E9006CDE0CB
:10264F00C3957350099006CEE0D395735002800264
:10265F00D22D9006CDE0D3957350099006CEE0C3EE
:10266F0095735002C22D9006CCE0B401099000E0A2
:10267F00E0D3956150028002C22D802A9006CDE0F2
:10268F00D3957340099006CEE0C395734002800244
:10269F00C22D9006CDE0C3957340099006CEE0D3CE
:1026AF0095734002D22D229006D0E09038B9F828C9
:1026BF002873804C85537380479000D4E0855FF07A
:1026CF00A4FFAEF074081200398F738033856173E5
:1026DF00802E856773802985687380248569738050
:1026EF001F856A73801A856B7380158566738010DA
:1026FF00856573800B856C73800690001AE0F57307
:1038B9000226C10226C30226C80226DC0226E1022C
:1038C90026E60226EB0226F00226F50226FA022651
:0738D900FF0227040227098A
:10270F009006D1E0FE9006D2E0D39E404B9006D0CB
:10271F00E0B404189006D2E0C395735002D22E9005
:10272F0006D1E0D395734002C22E802A9006D1E0E5
:10273F00C3957350099006D2E0D39573500280026F
:10274F00D22E9006D1E0D3957350099006D2E0C3F4
:10275F0095735002C22E802A9006D1E0D395734014
:10276F00099006D2E0C3957340028002C22E9006F4
:10277F00D1E0C3957340099006D2E0D39573400220
:10278F00D22E229006D4E09038E0F8282873804C9F
:10279F0085537380479000D4E0855FF0A4FFAEF0BF
:1027AF0074081200398F738033856173802E8567AB
:1027BF007380298568738024856973801F856A7388
:1027CF00801A856B7380158566738010856573809D
:0C27DF000B856C73800690001AE0F57307
:1038E00002279D02279F0227A40227B80227BD02B4
:1038F00027C20227C70227CC0227D10227D60227D8
:07390000DB0227E00227E5CE
:1027EB009006D5E0FE9006D6E0D39E404B9006D4E3
:1027FB00E0B404189006D6E0C395735002D22F9024
:10280B0006D5E0D395734002C22F802A9006D5E0FF
:10281B00C3957350099006D6E0D39573500280028E
:10282B00D22F9006D5E0D3957350099006D6E0C30E
:10283B0095735002C22F802A9006D5E0D395734032
:10284B00099006D6E0C3957340028002C22F900612
:10285B00D5E0C3957340099006D6E0D3957340023B
:10286B00D22F229006D8E0903907F8282873804C95
:10287B0085537380479000D4E0855FF0A4FFAEF0E2
:10288B0074081200398F738033856173802E8567CE
:10289B007380298568738024856973801F856A73AB
:1028AB00801A856B738015856673801085657380C0
:0C28BB000B856C73800690001AE0F5732A
:1039070002287902287B022880022894022899023B
:10391700289E0228A30228A80228AD0228B202285E
:07392700B70228BC0228C111
:1028C7009006D9E0FE9006DAE0D39E404B9006D8FA
:1028D700E0B404189006DAE0C395735002D2309042
:1028E70006D9E0D395734002C230802A9006D9E01A
:1028F700C3957350099006DAE0D3957350028002AE
:10290700D2309006D9E0D3957350099006DAE0C328
:1029170095735002C230802A9006D9E0D395734050
:10292700099006DAE0C3957340028002C230900630
:10293700D9E0C3957340099006DAE0D39573400256
:10294700D230229006DCE090392EF8282873804C8C
:1029570085537380479000D4E0855FF0A4FFAEF005
:1029670074081200398F738033856173802E8567F1
:102977007380298568738024856973801F856A73CE
:10298700801A856B738015856673801085657380E3
:0C2997000B856C73800690001AE0F5734D
:10392E0002295502295702295C02297002297502C3
:10393E00297A02297F02298402298902298E0229E5
:07394E009302299802299D54
:1029A3009006DDE0FE9006DEE0D39E404B9006DC11
:1029B300E0B404189006DEE0C395735002D2319060
:1029C30006DDE0D395734002C231802A9006DDE034
:1029D300C3957350099006DEE0D3957350028002CD
:1029E300D2319006DDE0D3957350099006DEE0C343
:1029F30095735002C231802A9006DDE0D39573406F
:102A0300099006DEE0C3957340028002C23190064E
:102A1300DDE0C3957340099006DEE0D39573400271
:102A2300D231229006E0E0903955F8282873804C83
:102A330085537380479000D4E0855FF0A4FFAEF028
:102A430074081200398F738033856173802E856714
:102A53007380298568738024856973801F856A73F1
:102A6300801A856B73801585667380108565738006
:0C2A73000B856C73800690001AE0F57370
:10395500022A31022A33022A38022A4C022A51024B
:103965002A56022A5B022A60022A65022A6A022A6C
:073975006F022A74022A7997
:102A7F009006E1E0FE9006E2E0D39E404B9006E028
:102A8F00E0B404189006E2E0C395735002D232907E
:102A9F0006E1E0D395734002C232802A9006E1E04E
:102AAF00C3957350099006E2E0D3957350028002EC
:102ABF00D2329006E1E0D3957350099006E2E0C35D
:102ACF0095735002C232802A9006E1E0D39573408D
:102ADF00099006E2E0C3957340028002C23290066D
:102AEF00E1E0C3957340099006E2E0D3957340028D
:102AFF00D232229006E4E090397CF8282873804C7B
:102B0F0085537380479000D4E0855FF0A4FFAEF04B
:102B1F0074081200398F738033856173802E856737
:102B2F007380298568738024856973801F856A7314
:102B3F00801A856B73801585667380108565738029
:0C2B4F000B856C73800690001AE0F57393
:10397C00022B0D022B0F022B14022B28022B2D02D3
:10398C002B32022B37022B3C022B41022B46022BF3
:07399C004B022B50022B55DA
:102B5B009006E5E0FE9006E6E0D39E404B9006E43F
:102B6B00E0B404189006E6E0C395735002D233909C
:102B7B0006E5E0D395734002C233802A9006E5E068
:102B8B00C3957350099006E6E0D39573500280020B
:102B9B00D2339006E5E0D3957350099006E6E0C377
:102BAB0095735002C233802A9006E5E0D3957340AB
:102BBB00099006E6E0C3957340028002C23390068B
:102BCB00E5E0C3957340099006E6E0D395734002A8
:102BDB00D233229006E8E09039A3F8282873804C72
:102BEB0085537380479000D4E0855FF0A4FFAEF06F
:102BFB0074081200398F738033856173802E85675B
:102C0B007380298568738024856973801F856A7337
:102C1B00801A856B7380158566738010856573804C
:0C2C2B000B856C73800690001AE0F573B6
:1039A300022BE9022BEB022BF0022C04022C09025E
:1039B3002C0E022C13022C18022C1D022C22022C7A
:0739C30027022C2C022C311D
:102C37009006E9E0FE9006EAE0D39E404B9006E856
:102C4700E0B404189006EAE0C395735002D23490BA
:102C570006E9E0D395734002C234802A9006E9E082
:102C6700C3957350099006EAE0D39573500280022A
:102C7700D2349006E9E0D3957350099006EAE0C391
:102C870095735002C234802A9006E9E0D3957340C9
:102C9700099006EAE0C3957340028002C2349006A9
:102CA700E9E0C3957340099006EAE0D395734002C3
:102CB700D234229006ECE09039CAF8282873804C69
:102CC70085537380479000D4E0855FF0A4FFAEF092
:102CD70074081200398F738033856173802E85677E
:102CE7007380298568738024856973801F856A735B
:102CF700801A856B73801585667380108565738070
:0C2D07000B856C73800690001AE0F573D9
:1039CA00022CC5022CC7022CCC022CE0022CE502E8
:1039DA002CEA022CEF022CF4022CF9022CFE022D06
:0739EA0003022D08022D0D60
:102D13009006EDE0FE9006EEE0D39E404B9006EC6D
:102D2300E0B404189006EEE0C395735002D23590D8
:102D330006EDE0D395734002C235802A9006EDE09C
:102D4300C3957350099006EEE0D395735002800249
:102D5300D2359006EDE0D3957350099006EEE0C3AB
:102D630095735002C235802A9006EDE0D3957340E7
:102D7300099006EEE0C3957340028002C2359006C7
:102D8300EDE0C3957340099006EEE0D395734002DE
:102D9300D23522AE2EAF2F74F5D39F74019E400817
:102DA300782E126A7C022EB0752F01752E00AE525A
:102DB300AF53E546BE000DD39F40099000B6E0D364
:102DC300954740028023754700E546C39553F57345
:102DD3009000B9E0D395454008E5452573F5458056
:102DE300069000B9E0F54580020547900092E0D3D4
:102DF3009561401CE55FC395604015AE52AF53E546
:102E030046BE00039F50099000B7E0D395484002A7
:102E1300806E9007D2E0A852B80004955350037512
:102E23004A009007D2E0A852B8000BD3955340064E
:102E3300E5539007D2F0E54A7041E553C39546F553
:102E430073E573D3940540037573059000B8E0C32D
:102E530095455007E573C3954540028009E545C391
:102E63009573F54580069000B8E0F5459000B8E00D
:102E7300D3954540069000B8E0F5457548008002BB
:102E83000548E54A7016900092E0C39561500DE540
:102E9300462405A852B8000695534002800F9000BF
:102EA300A5E0F545754A0174789007D2F022AE2E5D
:102EB300AF2F74E9D39F74039E4008782E126A7C67
:102EC30002304F752F01752E00754532A236402A08
:102ED3007545199000A5E075F002A4FFAEF0E54733
:102EE300BE0006D39F4002D2360547754A03747865
:102EF3009007D2F075490002303EAE52AF53E5461B
:102F03006F4E700302303EE546BE000DD39F40096D
:102F13009000B6E0D395474002800F754700E54A1D
:102F2300C394035003754519800DE546C39553F5C6
:102F330073E5472573F547900092E0D39561400E02
:102F43009007D2E0A852B80007D395534002800CF3
:102F530005499000A5E0B54903754A00E54AB40365
:102F630006A20DB3B34002800A0549E549B43C0308
:102F7300754A02E54AB402299007D2E0A852B80084
:102F83000ED395534009E5539007D2F0754900904D
:102F93000092E0C39561500975490074789007D297
:102FA300F0E54A705A900092E0D39561401CE55FCA
:102FB300C395604015AE52AF53E546BE00039F5024
:102FC300099000B7E0D39548400280087548007522
:102FD300454B8028E553C39546F573E573D39405B4
:102FE3004003757305900092E0D395614008E5486E
:102FF3002573F5488006E5482406F548754900E53C
:103003004A7016900092E0C39561500DE546240581
:10301300A852B80006955340028003754A01E54A59
:10302300B4011875451905499000A5E0B549067521
:103033004A0275490074789007D2F0E54575F00AA5
:10304300A4FFAEF09007C3EEF0A3EFF022E56F907C
:1030530039F1F828287390008AE0700302327790E0
:1030630000C0E0B40102800302319290004DE0B54C
:103073005E02800302318F7E017F00E5BE126A2863
:10308300E5BD2FFF50010E8E5A8F5B7410126A2814
:10309300900078E08E048F05FF126A189007C7EC42
:1030A300F0A3EDF074FFBC00039D500B74FF900779
:1030B300C7F8E4F0E8A3F0E56B600FE56BC394FE9B
:1030C30050089000E6E06402600280649000D4E05F
:1030D300B40B1F9007C7E0FEA3E0FF74E7126A2852
:1030E300E56B8E048F05FF126A189007C7ECF0A3F7
:1030F300EDF09000D4E0D3940B40089000BCE06462
:10310300046002802B9007C7E0FEA3E0FF9007C98D
:10311300E0FCA3E0FDEFD39DEE9C400D126A74909A
:1031230007C7EEF0A3EFF080079007C7E4F0A3F022
:1031330090008AE0B4021E9007C7E0FEA3E0FF9070
:1031430007D3E02FFF50010E74011200399007C717
:10315300EEF0A3EFF09007C7E0FEA3E0FF9007D3E4
:10316300E0BE0008D39F4004D2398002B2399007F1
:10317300C8E09007D3F09000BCE064016006A23978
:10318300B3B3400280069007C8E0F55F023275D200
:10319300397E017F00E5BE126A28E5BD2FFF50018D
:1031A3000E8E5A8F5B7410126A28900078E08E049A
:1031B3008F05FF126A189007C7ECF0A3EDF0E56BDB
:1031C300600FE56BC394FE50089000E6E064026074
:1031D3000280649000D4E0B40B1F9007C7E0FEA305
:1031E300E0FF74E7126A28E56B8E048F05FF126A0D
:1031F300189007C7ECF0A3EDF09000D4E0D3940B44
:1032030040089000BCE064046002802B9007C7E094
:10321300FEA3E0FF9007C9E0FCA3E0FDEFD39DEE22
:103223009C400D126A749007C7EEF0A3EFF080077D
:103233009007C7E4F0A3F090008AE0B4021E900761
:10324300C7E0FEA3E0FF9007D3E02FFF50010E7409
:10325300011200399007C7EEF0A3EFF09007C8E022
:103263009007D3F09000BCE0640160069007C8E0CB
:10327300F55F8003755F00900086E07006756F014F
:1032830002305075BB18023845900086E070030287
:1032930033FD7E017F00E5BE126A28E5BD2FFF5096
:1032A300010E8E5A8F5B9000CCE0B4010F7E0F7F2E
:1032B300FFAC5AAD5B126A748E5A8F5B9000F1E0DB
:1032C300B40245AE5AAF5B900023E0FCA3E0FDEDF2
:1032D300D39FEC9E400A900023E55AF0A3E55BF0F0
:1032E300AE5AAF5B900025E0FCA3E0FDEFD39DEE6B
:1032F3009C400A900025E55AF0A3E55BF0AE5AAF77
:103303005B74041200398F619000F1E0704CAE5A87
:10331300AF5B900023E0FCA3E0FDEFD39DEE9C4068
:1033230009126A748E5A8F5B8006755B00755A00AA
:10333300AE5AAF5B7410126A28900075E08E048F4A
:1033430005FF126A188C5A8D5B74FFBC0009D39D6C
:103353004005855B6180037561FE9000BCE0B401AC
:103363000280030233FBA20DB3B3500E900090E032
:10337300A852B80005D39553500280719000CDE058
:103383008561F0A4FFAEF074648E048F05FF126AAA
:10339300188C5A8D5BE56B6016E56BC394FE500F7A
:1033A3009000E6E0B402089000D4E0640B60028071
:1033B30017AE5AAF5B74E7126A28E56B8E048F056C
:1033C300FF126A188C5A8D5BAE5AAF5B9007C7E049
:1033D300FCA3E0FDEDD39FEC9E4005855B5F800B76
:1033E300A239B340069007C8E0F55F800BA239B35A
:1033F30040069007C8E0F55F80037561009000897F
:10340300E07006756F0202305075BB1902384590A3
:103413000089E070030234B2E55ED39551400302A4
:1034230034B0900021E0FEA3E0FFE565126A6C90E2
:103433000021EEF0A3EFF07E017F00E5BE126A28C3
:10344300E5BD2FFF50010E8E5A8F5B9000F6E070A2
:1034530013740A126A2874518E048F05FF126A18B6
:103463008D658019AE5AAF5B740A126A288F048E79
:10347300057E017F95CDCCCD1269168F65E565D3A9
:1034830094644003756564900021E0FEA3E0FFE5CA
:10349300652FFF50010E900021EEF0A3EFF0900096
:1034A3008DE0048E048F05FF126A188D6580037505
:1034B30065329000D9E07006756F0302305075BB1A
:1034C300130238459000D9E0604A7E017F00E5BED3
:1034D300126A28E5BD2FFF50010E8E5A8F5B7404CC
:1034E3001200398F669000DBE08566F0A4FDACF036
:1034F3007464FF126A188D669000DAE08566F0A4A2
:10350300FFAEF074FF8E048F05FF126A18ED900072
:1035130074F08003756600900087E07006756F0491
:1035230002305075BB17023845900087E0B40102A2
:1035330080030235C07E017F00E5BE126A28E5BD27
:103543002FFF50010E8E5A8F5B9007D4E0601990C5
:1035530007D4E01490638812008CE493FC74019305
:10356300FDEDC39FEC9E400280069007D4E014F06B
:103573009007D4E0C394B3501DAE5AAF5B9007D409
:10358300E00490638812008CE493FC740193FDEFD4
:10359300C39DEE9C400280069007D4E004F09007A0
:1035A300D4E0FE9000ADE08E0088F0A4FFAEF0748E
:1035B300648E048F05FF126A188D67800375670098
:1035C300900088E07006756F0502305075BB1602D7
:1035D3003845900088E0B4010280030236697E0119
:1035E3007F00E5BE126A28E5BD2FFF50010E8E5AFB
:1035F3008F5B9007D5E060199007D5E0149064F2D3
:1036030012008CE493FC740193FDEDC39FEC9E4088
:103613000280069007D5E014F09007D5E0C394B379
:10362300501DAE5AAF5B9007D5E0049064F21200D0
:103633008CE493FC740193FDEFC39DEE9C400280E8
:10364300069007D5E004F09007D5E0FE9000B3E0C4
:103653008E0088F0A4FFAEF074648E048F05FF1211
:103663006A188D68800375680075BB1F0238457E34
:10367300017F00E5BE126A28E5BD2FFF50010E8EC3
:103683005A8F5B7409126A2874E68E048F05FF1241
:103693006A188D6A90008FE07006756F07023050CC
:1036A30075BB1502384590008FE070030237C47E66
:1036B300017F00E5BE126A28E5BD2FFF50010E8E83
:1036C3005A8F5B74041200398F6990008FE0B40144
:1036D300159000E3E08569F0A4FFAEF074071200D3
:1036E30039EF9007CCF090008FE0B402159000E31F
:1036F300E08569F0A4FFAEF07407120039EF90077C
:10370300CBF090008FE0B4030280030237A7900050
:10371300D0E0701CE569C394195002D22BE569D33C
:1037230094644002C22B9000AFE09007CFF0806317
:103733009000AFE070349000E3E08569F0A4FFAE41
:10374300F074FF8E048F05FF126A18ED9007CFF017
:10375300AE52AF53741EBE0006D39F4002D22BE578
:1037630061D394E54002C22B8029E569C3940A50D2
:103773000DAE52AF53741EBE0004D39F500280029D
:10378300D22BE561D394E54002C22B9000AFE090C9
:1037930007CFF09007CFE0C3940550067405900758
:1037A300CFF0C23A90008FE0B40414E569C39419D2
:1037B3005002D23AE569D394324002C23AC22B8016
:1037C300037569009000E6E07006756F08023050DB
:1037D30075BB14806D9000E6E060567E017F00E5C6
:1037E300BE126A28E5BD2FFF50010E8E5A8F5BEF84
:1037F300D39421EE940E4005756BFF8015AE5AAF3E
:103803005B7410126A2874E38E048F05FF126A1822
:103813008D6BE56B75F00BA4FFAEF09000D4E08EDA
:10382300048F05FF126A189007C9ECF0A3EDF0802E
:1038330003756B0090008AE0600575BB1A80037501
:02384300BB18B0
:1039F10002305902328C0234120234C702352C02D1
:0B3A010035D50236720236A90237D814
:05384500056FD2EC222A
:096A5A002582F582500205832219
:0F008C0025E050020583258250020583F582226C
:1069F700EF2F500205832582F582E5833E2EF5832E
:016A0700226C
:106A6C00CFC39FFF50011E22C3EF9DFFEE9CFE2261
:086A7C000806B600021806220C
:0D6A3600A3E004F07006120049E004F02215
:0E003900048007C3CE13CECF13CFD5E0F6223E
:10691600BC000FBE0008ED8FF084FFADF022E4FE50
:10692600FF22BE000DEF60FE54F0606F20E7030209
:1069360069CCEAC0E0EBC0E078017A0075F001EEC0
:1069460020E710EF25E0FFEE33FE0AC5F023C5F081
:1069560030E7F0EA5407F9096A7A007B006001081B
:10696600C3EC9E40167004ED9F4010ED9FFDEC9E1B
:10697600FCE5F0CA4ACA03F5F08005E5F003F5F038
:10698600C3EE13FEEF13FFD9D77908CACBCAD8D006
:10699600EAFEEBFFD0E0FBD0E0FA22EC8FF084FCBD
:1069A600ED54F045F0C48FF084FEEDC454F045F08C
:1069B600C48FF084FDEEC4FE54F02DFFEE540F3C60
:1069C600FEADF07C0022790078008FF0EC7E082086
:1069D600E70DC3CD33CD33C933C9C833C8DEF08420
:1069E60049F9E5F08FF0BE00E6FD7C00E9FFE8FE20
:0169F600227E
:0E6A2800F88FF0A4FFE5F0CE88F0A42EFE2239
:10000300EF8DF0A4F9A8F0EF8CF0A428F8EE8DF0B2
:06001300A428FEE9FF2213
:106A0800600D782B026A12007830D8FED5E0F822A3
:106A1800EEC0E07E00126916EFFDEEFCD0E0FE222B
:0C6A4300EEC0E07E00126916D0E0FE22DA
:03001B0002001EC2
:0300530002005652
:03009B00020071EF
:03000000026A632E
:096A630075817575D0000244C96B
:0B6A4F00E5822FF582E5833EF58322EF
:0A0049000582D5820215831582227C
:10001E00C0E0C0F0C083C082C0D075D0001244488A
:0B002E00D0D0D082D083D0F0D0E032E0
:10005600C0E0C0F0C083C082C0D075D00012444B4F
:10006600D0D0D082D083D0F0D0E032C0E0C0F0C093
:1000760083C082C0D075D000124467D0D0D082D061
:0600860083D0F0D0E0324F
:00000001FF
